:020000040800F2
:1000000000500020255B0008DD910008E191000808
:10001000E5910008E9910008ED910008000000005A
:10002000000000000000000000000000F191000846
:10003000F591000800000000F9910008FD9100080A
:10004000715B0008715B0008715B0008715B000860
:10005000715B0008715B0008715B0008715B000850
:10006000715B0008715B0008715B00088541000846
:10007000715B0008715B0008715B0008715B000830
:10008000715B0008715B0008E9400008715B0008C3
:10009000715B0008715B0008715B0008715B000810
:1000A000715B0008715B0008715B0008753F000818
:1000B000715B0008715B0008715B0008715B0008F0
:1000C000715B0008715B0008715B0008715B0008E0
:1000D000715B000841920008715B0008715B0008C9
:1000E000715B0008715B0008715B00080000000094
:1000F0000000000000000000000000000000000000
:0C01000000000000000000005FF808F1A3
:10011000830770B5064614D10368A3F1013222EAC1
:10012000030313F0803F0CD1031D1A4653F8044B10
:10013000A4F1013525EA040414F0803FF5D01046FF
:1001400000E0304603782BB1431C18460133047895
:10015000002CFAD100F002F8304670BD80EA0102AE
:10016000844612F0030F4FD111F0030F32D14DF836
:10017000044D11F0040F51F8043B0BD0A3F10132F0
:100180009A4312F0803F04BF4CF8043B51F8043B03
:1001900016D100BF51F8044BA3F101329A4312F07B
:1001A000803FA4F101320BD14CF8043BA24312F082
:1001B000803F04BF51F8043B4CF8044BEAD023467F
:1001C0000CF8013B13F0FF0F4FEA3323F8D15DF831
:1001D000044B704711F0010F06D011F8012B0CF8F9
:1001E000012B002A08BF704711F0020FBFD031F871
:1001F000022B12F0FF0F16BF2CF8022B8CF80020F8
:1002000012F47F4FB3D1704711F8012B0CF8012B7A
:10021000002AF9D1704700BF20F0030110F003005D
:10022000C0F1000051F8043B00F1040C4FEACC0C83
:100230006FF000021CBF22FA0CF213434FF0010CC6
:100240004CEA0C2C4CEA0C4CA3EB0C0222EA030205
:1002500012EACC1204BF51F8043B0430F4D013F07E
:10026000FF0F1FBF013013F47F4F013013F47F0FD6
:1002700018BF0130704700BF2DE9F0478AB004462F
:100280000D4600F04FF840F2000AC2F2000A9AF957
:100290000030013306460F460FD02046294600F0B5
:1002A00007F950B14FF000084FF0000920462946E9
:1002B00042464B4600F056FD20B9304639460AB05A
:1002C000BDE8F0879AF800604CF2F403C0F6000332
:1002D0000122CDE904458DE80C000023CDE902455B
:1002E000089356B9CDE90689684600F009F970B15E
:1002F000089B8BB9DDE90667DFE740464946424681
:100300004B4600F0E7FB022ECDE90601ECD100F0F0
:10031000F9F821230360EBE700F0F4F8089B036091
:10032000E8E700BF2DE9F8430027B946C7F6F077A4
:10033000C7F6F0790F404F4504460D4602460B467E
:100340000E46804600F09980002977DD0F1500F0F9
:10035000828026F07F43A7F2FF3723F47003FA0769
:1003600043F4801344BF4FEAD8724FEA48084FF075
:10037000000C48BF02EB430360464FEAD8727F107F
:1003800002EB430316244FEA48024FF400114518CC
:10039000D60F9D424FEA4202DEBFC5EB0303681849
:1003A0008C444908013C06EB4303F0D12026A046CB
:1003B0004FF000410EE081461B1A954288BF013B79
:1003C000521B64184846D50F49085200013E05EB00
:1003D000430315D0984201EB080503DB954298BF13
:1003E0008342F0D105F0004905EB0108B9F1004F57
:1003F000E1D1B8F1000FA8BF00F10109DCDADAE7BA
:10040000134312D166084FEA6C031CF0010F03F18D
:100410007F5318BF46F0004603F50013344603EB44
:10042000075520462946BDE8F883631C08BF0CF138
:10043000010CE8D004F001031C19E3E721F00046A9
:100440000643EED041BB0F464FEAD826153F4FEA90
:100450004858002EF8D016F4801319D176000133D5
:10046000F102FBD5C3F10101C3F1200228FA02F227
:100470007F18164308FA03F86BE700F001FA02460A
:100480000B462046294600F049F804460D46C8E7C9
:10049000202201210023E9E702460B4600F03CF848
:1004A00002460B4600F016FB04460D46B9E700BFB6
:1004B00050EA010201D102207047D0F1010238BF99
:1004C0000022B1F1004F08BF0028F4D021F0004312
:1004D0004FF6FF71A3F58010C7F6DF71884201D88F
:1004E00004207047B3F5801F01D20320704700201D
:1004F000C7F6F070834214BF002002F0010070477D
:100500000020704740F20403C2F2000318687047ED
:1005100081F0004102E000BF83F0004330B54FEAB4
:1005200041044FEA430594EA050F08BF90EA020F21
:100530001FBF54EA000C55EA020C7FEA645C7FEAB4
:10054000655C00F0E2804FEA5454D4EB5555B8BFD7
:100550006D420CDD2C4480EA020281EA030382EA48
:10056000000083EA010180EA020281EA0303362DDA
:1005700088BF30BD11F0004F4FEA01314FF4801CAD
:100580004CEA113102D0404261EB410113F0004FBF
:100590004FEA03334CEA133302D0524263EB430376
:1005A00094EA050F00F0A780A4F10104D5F1200E14
:1005B0000DDB02FA0EFC22FA05F2801841F100016F
:1005C00003FA0EF2801843FA05F359410EE0A5F143
:1005D00020050EF1200E012A03FA0EFC28BF4CF074
:1005E000020C43FA05F3C01851EBE37101F000452A
:1005F00007D54FF0000EDCF1000C7EEB00006EEB37
:100600000101B1F5801F1BD3B1F5001F0CD34908C0
:100610005FEA30004FEA3C0C04F101044FEA445217
:1006200012F5800F80F09A80BCF1004F08BF5FEA9E
:10063000500C50F1000041EB045141EA050130BD7E
:100640005FEA4C0C404141EB010111F4801FA4F121
:100650000104E9D191F0000F04BF01460020B1FA76
:1006600081F308BF2033A3F10B03B3F120020CDAAE
:100670000C3208DD02F1140CC2F10C0201FA0CF08C
:1006800021FA02F10CE002F11402D8BFC2F1200CF1
:1006900001FA02F120FA0CFCDCBF41EA0C019040A7
:1006A000E41AA2BF01EB0451294330BD6FEA0404F0
:1006B0001F3C1CDA0C340EDC04F11404C4F12002DB
:1006C00020FA04F001FA02F340EA030021FA04F3ED
:1006D00045EA030130BDC4F10C04C4F1200220FA44
:1006E00002F001FA04F340EA0300294630BD21FA82
:1006F00004F0294630BD94F0000F83F4801306BF48
:1007000081F480110134013D4EE77FEA645C18BF3B
:100710007FEA655C29D094EA050F08BF90EA020FD2
:1007200005D054EA000C04BF1946104630BD91EACA
:10073000030F1EBF0021002030BD5FEA545C05D1CD
:100740004000494128BF41F0004130BD14F580040C
:100750003CBF01F5801130BD01F0004545F0FE4180
:1007600041F470014FF0000030BD7FEA645C1ABFB5
:10077000194610467FEA655C1CBF0B46024650EAEC
:10078000013406BF52EA033591EA030F41F4002118
:1007900030BD00BF90F0000F04BF0021704730B59E
:1007A0004FF4806404F132044FF000054FF0000173
:1007B00050E700BF90F0000F04BF0021704730B534
:1007C0004FF4806404F1320410F0004548BF404209
:1007D0004FF000013EE700BF42004FEAE2014FEA5E
:1007E00031014FEA02701FBF12F07F4393F07F4F39
:1007F00081F06051704792F0000F14BF93F07F4F6B
:10080000704730B54FF4607401F0004521F00041AD
:1008100020E700BF50EA010208BF704730B54FF033
:1008200000050AE050EA010208BF704730B511F038
:10083000004502D5404261EB41014FF4806404F170
:1008400032045FEA915C3FF4DCAE4FF003025FEAF2
:10085000DC0C18BF03325FEADC0C18BF033202EB7A
:10086000DC02C2F1200300FA03FC20FA02F001FAD4
:1008700003FE40EA0E0021FA02F11444C1E600BF73
:1008800070B54FF0FF0C4CF4E06C1CEA11541DBF26
:100890001CEA135594EA0C0F95EA0C0F00F0DEF8F1
:1008A0002C4481EA030621EA4C5123EA4C5350EAD6
:1008B000013518BF52EA033541F4801143F4801327
:1008C00038D0A0FB02CE4FF00005E1FB02E506F0B8
:1008D0000042E0FB03E54FF00006E1FB03569CF00D
:1008E000000F18BF4EF0010EA4F1FF04B6F5007F13
:1008F00064F5407404D25FEA4E0E6D4146EB060685
:1009000042EAC62141EA55514FEAC52040EA5E500D
:100910004FEACE2EB4F1FD0C88BFBCF5E06F1ED8B7
:10092000BEF1004F08BF5FEA500E50F1000041EBEE
:10093000045170BD06F0004646EA010140EA02009B
:1009400081EA0301B4EB5C04C2BFD4EB0C0541EABD
:10095000045170BD41F480114FF0000E013C00F3D2
:10096000AB8014F1360FDEBF002001F0004170BDF6
:10097000C4F10004203C35DA0C341BDC04F114040F
:10098000C4F1200500FA05F320FA04F001FA05F29B
:1009900040EA020001F0004221F0004110EBD37068
:1009A00021FA04F642EB06015EEA430E08BF20EA94
:1009B000D37070BDC4F10C04C4F1200500FA04F337
:1009C00020FA05F001FA04F240EA020001F00041C9
:1009D00010EBD37041F100015EEA430E08BF20EA3C
:1009E000D37070BDC4F1200500FA05F24EEA020E84
:1009F00020FA04F301FA05F243EA020321FA04F0B3
:100A000001F0004121FA04F220EA020000EBD37069
:100A10005EEA430E08BF20EAD37070BD94F0000F69
:100A20000FD101F00046400041EB010111F4801F9D
:100A300008BF013CF7D041EA060195F0000F18BF4E
:100A4000704703F00046520043EB030313F4801F8A
:100A500008BF013DF7D043EA0603704794EA0C0F44
:100A60000CEA135518BF95EA0C0F0CD050EA41065A
:100A700018BF52EA4306D1D181EA030101F00041D7
:100A80004FF0000070BD50EA410606BF10461946FF
:100A900052EA430619D094EA0C0F02D150EA01360B
:100AA00013D195EA0C0F05D152EA03361CBF10464C
:100AB00019460AD181EA030101F0004141F0FE41EB
:100AC00041F470014FF0000070BD41F0FE4141F46F
:100AD000780170BD70B54FF0FF0C4CF4E06C1CEA6F
:100AE00011541DBF1CEA135594EA0C0F95EA0C0F24
:100AF00000F0A7F8A4EB050481EA030E52EA0335DF
:100B00004FEA013100F088804FEA03334FF08055FF
:100B100045EA131343EA12634FEA022245EA11152C
:100B200045EA10654FEA00260EF000419D4208BFDD
:100B3000964244F1FD0404F5407402D25B084FEA8A
:100B40003202B61A65EB03055B084FEA32024FF436
:100B500080104FF4002CB6EB020E75EB030E22BF93
:100B6000B61A754640EA0C005B084FEA3202B6EB53
:100B7000020E75EB030E22BFB61A754640EA5C0002
:100B80005B084FEA3202B6EB020E75EB030E22BF92
:100B9000B61A754640EA9C005B084FEA3202B6EB93
:100BA000020E75EB030E22BFB61A754640EADC0052
:100BB00055EA060E18D04FEA051545EA16754FEAB4
:100BC00006164FEAC30343EA52734FEAC2025FEAD2
:100BD0001C1CC0D111F4801F0BD141EA00014FF061
:100BE00000004FF0004CB6E711F4801F04BF014332
:100BF0000020B4F1FD0C88BFBCF5E06F3FF6AFAE4E
:100C0000B5EB030C04BFB6EB020C5FEA500C50F1DD
:100C1000000041EB045170BD0EF0004E4EEA113160
:100C200014EB5C04C2BFD4EB0C0541EA045170BD67
:100C300041F480114FF0000E013C90E645EA060EAB
:100C40008DE60CEA135594EA0C0F08BF95EA0C0FD9
:100C50003FF43BAF94EA0C0F0AD150EA01347FF421
:100C600034AF95EA0C0F7FF425AF104619462CE7F8
:100C700095EA0C0F06D152EA03353FF4FDAE10465B
:100C8000194622E750EA410618BF52EA43067FF4AC
:100C9000C5AE50EA41047FF40DAF52EA43057FF43C
:100CA000EBAE12E74FF0FF3C06E000BF4FF0010C47
:100CB00002E000BF4FF0010C4DF804CD4FEA410CAB
:100CC0007FEA6C5C4FEA430C18BF7FEA6C5C1BD078
:100CD00001B050EA410C0CBF52EA430C91EA030FF9
:100CE00002BF90EA020F0020704710F1000F91EA56
:100CF000030F58BF994208BF90422CBFD8176FEA24
:100D0000E37040F0010070474FEA410C7FEA6C5CF1
:100D100002D150EA013C07D14FEA430C7FEA6C5CF8
:100D2000D6D152EA033CD3D05DF8040B704700BF24
:100D30008446104662468C461946634600E000BF72
:100D400001B5FFF7B7FF002848BF10F1000F01BD44
:100D50004DF808EDFFF7F4FF0CBF012000205DF80F
:100D600008FB00BF4DF808EDFFF7EAFF34BF012094
:100D700000205DF808FB00BF4DF808EDFFF7E0FF2D
:100D800094BF012000205DF808FB00BF4DF808ED7E
:100D9000FFF7CEFF94BF012000205DF808FB00BFE5
:100DA0004DF808EDFFF7C4FF34BF012000205DF8C7
:100DB00008FB00BF4FEA410212F5001215D211D50F
:100DC0006FF47873B3EB625212D94FEAC12343F048
:100DD000004343EA505311F0004F23FA02F018BFCA
:100DE000404270474FF00000704750EA013005D193
:100DF00011F0004008BF6FF0004070474FF0000056
:100E0000704700BF4FEA4102B2F1E04324BFB3F59F
:100E1000001CDCF1FE5C0DD901F0004C4FEAC00271
:100E20004CEA5070B2F1004F40EB830008BF20F055
:100E30000100704711F0804F21D113F13872BCBF0F
:100E400001F00040704741F480114FEA5252C2F164
:100E50001802C2F1200C10FA0CF320FA02F018BFAD
:100E600040F001004FEAC1234FEAD32303FA0CFC00
:100E700040EA0C0023FA02F34FEA4303CCE77FEA8F
:100E8000625307D150EA01331EBF4FF0FE4040F4D9
:100E90004000704701F0004040F0FE4040F4000088
:100EA000704700BF80F0004002E000BF81F00041C9
:100EB00042001FBF5FEA410392EA030F7FEA226C00
:100EC0007FEA236C6AD04FEA1262D2EB1363C1BF90
:100ED000D218414048404140B8BF5B42192B88BFFF
:100EE000704710F0004F40F4000020F07F4018BF22
:100EF000404211F0004F41F4000121F07F4118BF42
:100F0000494292EA030F3FD0A2F1010241FA03FCE9
:100F100010EB0C00C3F1200301FA03F100F00043D1
:100F200002D5494260EB4000B0F5000F13D3B0F199
:100F3000807F06D340084FEA310102F10102FE2A08
:100F400051D2B1F1004F40EBC25008BF20F0010078
:100F500040EA03007047490040EB000010F4000F26
:100F6000A2F10102EDD1B0FA80FCACF1080CB2EBB9
:100F70000C0200FA0CF0AABF00EBC2505242184318
:100F8000BCBFD0401843704792F0000F81F40001BD
:100F900006BF80F400000132013BB5E74FEA410390
:100FA0007FEA226C18BF7FEA236C21D092EA030FFC
:100FB00004D092F0000F08BF0846704790EA010F76
:100FC0001CBF0020704712F07F4F04D1400028BFA3
:100FD00040F00040704712F100723CBF00F5000085
:100FE000704700F0004343F0FE4040F400007047BB
:100FF0007FEA226216BF08467FEA23630146420267
:1010000006BF5FEA412390EA010F40F48000704779
:101010004FF0000304E000BF10F0004348BF40421F
:101020005FEA000C08BF704743F0964301464FF05B
:1010300000001CE050EA010208BF70474FF00003B7
:101040000AE000BF50EA010208BF704711F00043F8
:1010500002D5404261EB41015FEA010C02BF8446C8
:101060000146002043F0B64308BFA3F18053A3F527
:101070000003BCFA8CF2083AA3EBC25310DB01FA6E
:1010800002FC634400FA02FCC2F12002BCF1004FF2
:1010900020FA02F243EB020008BF20F00100704783
:1010A00002F1200201FA02FCC2F1200250EA4C00D7
:1010B00021FA02F243EB020008BF20EADC7070471D
:1010C0004FF0FF0C1CEAD0521EBF1CEAD15392EA2B
:1010D0000C0F93EA0C0F6FD01A4480EA010C400207
:1010E00018BF5FEA41211ED04FF0006343EA501061
:1010F00043EA5111A0FB01310CF00040B1F5000FA3
:101100003EBF490041EAD3715B0040EA010062F151
:101110007F02FD2A1DD8B3F1004F40EBC25008BF3B
:1011200020F00100704790F0000F0CF0004C08BF59
:1011300049024CEA502040EA51207F3AC2BFD2F126
:10114000FF0340EAC250704740F400004FF0000334
:10115000013A5DDC12F1190FDCBF00F0004070476E
:10116000C2F10002410021FA02F1C2F1200200FAAC
:1011700002FC5FEA310040F1000053EA4C0308BF73
:1011800020EADC70704792F0000F00F0004C02BFC4
:10119000400010F4000F013AF9D040EA0C0093F03F
:1011A000000F01F0004C02BF490011F4000F013B99
:1011B000F9D041EA0C018FE70CEAD15392EA0C0F07
:1011C00018BF93EA0C0F0AD030F0004C18BF31F072
:1011D000004CD8D180EA010000F00040704790F048
:1011E000000F17BF90F0004F084691F0000F91F0EC
:1011F000004F14D092EA0C0F01D142020FD193EAB2
:101200000C0F03D14B0218BF084608D180EA010039
:1012100000F0004040F0FE4040F40000704740F015
:10122000FE4040F4400070474FF0FF0C1CEAD052E3
:101230001EBF1CEAD15392EA0C0F93EA0C0F69D03F
:10124000A2EB030280EA010C49024FEA402037D0AA
:101250004FF0805343EA111143EA10130CF00040A1
:101260008B4238BF5B0042F17D024FF4000C8B4291
:1012700024BF5B1A40EA0C00B3EB510F24BFA3EB71
:10128000510340EA5C00B3EB910F24BFA3EB910341
:1012900040EA9C00B3EBD10F24BFA3EBD10340EA9B
:1012A000DC001B0118BF5FEA1C1CE0D1FD2A3FF6E1
:1012B00050AF8B4240EBC25008BF20F00100704796
:1012C0000CF0004C4CEA50207F32C2BFD2F1FF0339
:1012D00040EAC250704740F400004FF00003013A6A
:1012E00037E792F0000F00F0004C02BF400010F40E
:1012F000000F013AF9D040EA0C0093F0000F01F022
:10130000004C02BF490011F4000F013BF9D041EA43
:101310000C0195E70CEAD15392EA0C0F08D1420276
:101320007FF47DAF93EA0C0F7FF470AF084676E749
:1013300093EA0C0F04D14B023FF44CAF08466EE722
:1013400030F0004C18BF31F0004CCAD130F00042F0
:101350007FF45CAF31F000437FF43CAF5FE700BF48
:101360004FF0FF3C06E000BF4FF0010C02E000BF71
:101370004FF0010C4DF804CD4FEA40024FEA410313
:101380007FEA226C18BF7FEA236C11D001B052EAC9
:10139000530C18BF90EA010F58BFB2EB030088BF8F
:1013A000C81738BF6FEAE17018BF40F001007047FE
:1013B0007FEA226C02D15FEA402C05D17FEA236CE0
:1013C000E4D15FEA412CE1D05DF8040B704700BF27
:1013D000844608466146FFE70FB5FFF7C9FF0028BE
:1013E00048BF10F1000F0FBD4DF808EDFFF7F4FFF7
:1013F0000CBF012000205DF808FB00BF4DF808ED90
:10140000FFF7EAFF34BF012000205DF808FB00BFB2
:101410004DF808EDFFF7E0FF94BF012000205DF8D4
:1014200008FB00BF4DF808EDFFF7D2FF94BF012085
:1014300000205DF808FB00BF4DF808EDFFF7C8FF7E
:1014400034BF012000205DF808FB00BF42000ED22F
:10145000B2F1FE4F0BD34FF09E03B3EB126209D4EF
:101460004FEA002343F0004323FA02F070474FF0A5
:101470000000704712F1610F01D1420202D14FF01A
:10148000FF3070474FF00000704700BF00000000C1
:1014900090B585B002AF041C081C111C1A1CBB1DA2
:1014A0001C803B1D1880BB1C19803B1C1A80BB1C78
:1014B0001B88013B1B041B0C1B041B0CBA1D0020CA
:1014C000115E3A1D0020125E1B041B14381C1830DC
:1014D00000880090081C111C1A1C012305F0BCFF99
:1014E0003B1D1A883B1C1B88D3181B041B0C013B9B
:1014F0001B041B0C1B041B0CBA1D0020115E1B04DB
:101500001B14BA1C0020125E381C18300088009092
:10151000081C191C012305F09FFF3B1C1B88013B85
:101520001B041B0C1B041B0CBA1D0020115E3A1D72
:101530000020125E1B041B14381C18300088009019
:10154000081C111C012205F087FFBB1D1A88BB1C5B
:101550001B88D3181B041B0C013B1B041B0C1B0416
:101560001A0C3B1C1B88013B1B041B0C1B041B0C93
:1015700012041214391D0020095E1B041B14381CB0
:10158000183000880090101C012205F065FFBD4650
:1015900003B090BC01BC004780B500AF214B802256
:1015A0001A80204B00229A801E4B17221A811D4B55
:1015B00000229A811B4B00221A821A4B00229A8227
:1015C000184B194A1A83174B00229A83154A174B56
:1015D0001B681B041B0C1384124B00229A84114BB2
:1015E00000221A850F4B012252429A850D4B104A58
:1015F0009A860C4B02221A870A4B00229A87094AC4
:1016000040230021D152074A48230021D152054AE4
:101610004C230021D152034B81221A80BD4680BC4D
:1016200001BC0047002C014001300000B81D002023
:101630008813000080B500AF8023DB0580221A806C
:101640008023DB0550229A808023DB0500221A814B
:101650008023DB0500229A818023DB0500221A8289
:101660008023DB0500229A828023DA051D4B1B684C
:101670001B041B0C13838023DB0500229A83802329
:10168000DB0510221A848023DB0500229A84802344
:10169000DB0508221A858023DB0509229A85802331
:1016A000DB05114A9A868023DB0505221A878023F1
:1016B000DB0500229A878023DA0540230021D152DE
:1016C0008023DA0548230021D1528023DA054C23F8
:1016D0000021D1528023DB0580221A80BD4680BCC8
:1016E00001BC0047BC1D00208813000080B500AF7E
:1016F000214B00221A60204B00225A601E4B1F4AC9
:1017000012689A601C4B0022DA601B4B00221A619F
:10171000194B00225A61184B00229A61164B002285
:10172000DA61154B00221A62134B154A5A62124BAA
:1017300000229A62104B0022DA620F4B00221A63D9
:101740000D4B00225A630C4B00229A630A4B0A4A43
:10175000926804210A439A60C046074B9A680423A2
:101760001340FAD0044B044A926801210A439A605C
:10177000BD4680BC01BC004700240140C01D0020C4
:10178000FF0F000080B500AF084B094A128A5A606B
:10179000064B084A9A60054B074ADA60034B074A32
:1017A00012681A60BD4680BC01BC004708000240B8
:1017B000640400204C24014078040020C41D002053
:1017C00080B582B000AF80231B05181C002108F0F3
:1017D000ADF8BD4602B080BC01BC004780B58EB0FC
:1017E00002AF3B1C2E3303221A801AE03B1D03205C
:1017F00005211A1C02F00EFF031C18D03B1C2E33CF
:101800003A1C2E321288013A1A80704B181C01F0D3
:101810009FFE6E4B181C01F09BFE6C4B181C01F0D8
:1018200097FE3B1C2E331B88002BDFD100E0C04607
:101830003B1C2E331B88002B1CD13B1C2E330A2251
:101840001A800AE0614B181C01F082FE3B1C2E330B
:101850003A1C2E321288013A1A803B1C2E331B8808
:10186000002BEFD15A4B5A4AD268802109024A40D4
:10187000DA60E2E73A1D20230021D1543A1D554B8E
:1018800000210091544901911820D22105F00AFE4F
:10189000524B1B8A5B081B041B0C1B041A0C4F4B7E
:1018A000DA814F4B4F4A9A614D4B00225A804C4B84
:1018B00000221A714A4B00221A80484B5A88484B22
:1018C000DA80464B1B8A1B041A0C454B9A81464B07
:1018D000464A1A60464B434A1A603B1C2E33032289
:1018E0001A801AE0434B082005211A1C02F092FED0
:1018F000031C18D03B1C2E333A1C2E321288013A9E
:101900001A80324B181C01F023FE304B181C01F0DA
:101910001FFE2E4B181C01F01BFE3B1C2E331B8898
:10192000002BDFD100E0C0463B1C2E331B88002B70
:101930001CD13B1C2E330A221A800AE0234B181CB0
:1019400001F006FE3B1C2E333A1C2E321288013A5F
:101950001A803B1C2E331B88002BEFD11C4B1C4ADA
:10196000D268802109024A40DA60E2E7FFF714FEFC
:10197000FFF760FEFFF7BAFEFFF704FF3B1C2E33B4
:1019800000221A80174BBB6214E0144B1B891B0406
:101990001B0C802292009B181B041A0CBB6A1A8035
:1019A000BB6A0233BB623B1C2E333A1C2E321288B8
:1019B00001321A80094B1B8A3A1C2E3212889A4235
:1019C000E3D3BD460CB080BC01BC0047DCFF000087
:1019D00000080140FFFF0000040200206404002012
:1019E000DC1D0020A415002090210020A5F300009C
:1019F000FC1D0020A81D002080B582B000AF0A1C8D
:101A0000BB1D011C19803B1D1A80BA1D3B1D002106
:101A1000525E00215B5E9A4202DABB1D1B8801E028
:101A20003B1D1B881B041B14181CBD4602B080BC48
:101A300002BC084780B582B000AF0A1CBB1D011C68
:101A400019803B1D1A80BA1D3B1D0021525E0021EA
:101A50005B5E9A4202DDBB1D1B8801E03B1D1B88BB
:101A60001B041B14181CBD4602B080BC02BC0847F6
:101A700080B584B000AF021C3960BB1D1A80BB1D4D
:101A80001B88181C5C4903F0EFFD031C1B041A0C97
:101A90003B1C0F331A703B1C0F331B78302213434F
:101AA0001B061A0E3B681A703B1C0F331B781B0475
:101AB0001B0C1A1CD200D21A111C49018A1A1201DD
:101AC000D31A1B011B04190CBB1DBA1D12888A18DE
:101AD0001A80BB1D1B88181CFA23990003F0C4FD53
:101AE000031C1B041A0C3B1C0F331A703B68013398
:101AF0003A1C0F32127830210A431206120E1A7065
:101B00003B1C0F331B781B041B0C1A1C9201D21AAE
:101B10009201D2185200D318DB001B04190CBB1D14
:101B2000BA1D12888A181A80BB1D1B88181C6421D4
:101B300003F09AFD031C1B041A0C3B1C0F331A7094
:101B40003B6802333A1C0F32127830210A431206E6
:101B5000120E1A703B1C0F331B781B041B0C1A1C33
:101B60005202D21A9200D218D200D31A9B001B0440
:101B7000190CBB1DBA1D12888A181A80BB1D1B8840
:101B8000181C0A2103F070FD031C1B041A0C3B1CDB
:101B90000F331A703B6803333A1C0F32127830212E
:101BA0000A431206120E1A703B1C0F331B781B04DB
:101BB0001B0C1A1C5203D21A9200D31A5B001B048E
:101BC000190CBB1DBA1D12888A181A803B68043391
:101BD000BA1D12881206120E30210A431206120E86
:101BE0001A703B68053300221A703B68181CBD460A
:101BF00004B080BC02BC08471027000080B500AFCD
:101C00008023DB05144A127812061216511E134A5D
:101C100049008A5A013A1204120C1A858023DB0506
:101C20000D4A127812061216511E0D4A49008A5AA0
:101C3000013A1204120C9A858023DB058022D2051A
:101C4000928D1204120C52081204120C1A87BD460F
:101C500080BC01BC0047C046640400205C01002039
:101C60008C01002080B582B000AFA74B1B882B22CF
:101C700093431B041A0CA44B1A80A34B1B881A1CF9
:101C80000423134000D038E18023DB058022D205F5
:101C900012881204120C01218A431204120C1A80B9
:101CA0009A4B9A4A92891204120C06218A43120412
:101CB000120C9A81964B964A126801218A431A6047
:101CC000934B934A126806218A431A60914B914ABA
:101CD00052680F210A435A608F4B8F4A5268202165
:101CE0008A435A608C4B8C4A126802218A431A60DC
:101CF0008A4B1B781B061B160D2B0ADC874B9B7A25
:101D0000002B06D1824B864ADA607F4B844A5A61A7
:101D100005E07F4B834ADA607B4B824A5A617C4BF9
:101D20007E4A128A5A607A4B794A126804210A4321
:101D30001A60764B794A128A1A87744B734A9289D1
:101D40001204120C06218A431204120C9A816F4B62
:101D50006E4A128A1204120C06218A431204120CD3
:101D60001A826E4B1B781B061B160D2B0DDD6B4B61
:101D70009B7A002B09D1654B644A92891204120C9C
:101D800004210A431204120C9A81674B1B681A1C27
:101D9000664B9A4255D1644B614A1A60BB1D0322BF
:101DA0001A8018E0624B082005211A1C02F032FC50
:101DB000031C15D0BB1DBA1D1288013A1A805D4B59
:101DC000181C01F0C5FB5B4B181C01F0C1FB594B03
:101DD000181C01F0BDFBBB1D1B88002BE2D100E0ED
:101DE000C046BB1D1B88002B18D1BB1D0A221A80C0
:101DF00008E0504B181C01F0ABFBBB1DBA1D12884C
:101E0000013A1A80BB1D1B88002BF2D14A4B4A4A6B
:101E1000D268802109024A40DA60E6E7444B1A683A
:101E2000464B1A60464B1A68464B1A60464B1A6876
:101E3000464B1A60464B1A68464B1A60324BFF22DB
:101E40005A80FFF7DBFE354B1B781B061B160D2B4C
:101E500010DC324B9B7A002B0CD12F4B2E4A526850
:101E600020210A435A602C4B2B4A91683A4A0A4077
:101E70009A600CE0284B284A9268802149000A4366
:101E80009A60234B224A126801210A431A60234BAD
:101E9000DB7A1B061B16012B0AD11C4B1B4A128C2A
:101EA0001204120C02218A431204120C1A8409E053
:101EB000164B164A128C1204120C02210A43120409
:101EC000120C1A84104B00221A770F4B5B881022D9
:101ED00013431B041A0C0C4B5A800C4B00229A849F
:101EE0008023DB058022D20512881204120C012106
:101EF0000A431204120C1A8000E0C046BD4602B02C
:101F000080BC01BC0047C046DC1D0020002C014005
:101F10000800024000000240002401406404002048
:101F2000A41500207804002090210020A5F30000D3
:101F3000A81D0020DCFF00000008014060200020F8
:101F4000AC1D002094210020B01D00205C2000204A
:101F5000B41D00202C1F0020FFFEFFFFF0B54746F8
:101F600080B486B000AF924B802212021A61914B6E
:101F70001B881A1C0223134044D008E08D4B1A8A98
:101F80008D4B1B8AD31A1B041A0C8A4B1A82894B5D
:101F90001A8A894B1B8A9A42F0D2884BDA68864BA0
:101FA0001B8A191C844BDB891B041B14CB1A5B0096
:101FB000191C804B1B8A5B00CB18D3181A1C7D4B55
:101FC0005A617C4B5A697D4BD9687B4B1B8A5B00FD
:101FD000CB189A4208D3774B5A69774B1B8A5B0020
:101FE0005B42D218734B5A61734B9B7A1B061B16CC
:101FF000022B07D16F4B1B88202213431B041A0CA2
:102000006C4B1A806B4B1B881A1C0423134001D0A5
:1020100000F0B6FE684B1B781B061B16162B40DC27
:10202000644B5B697B61664B3B610023BB603B1C7F
:102030000E33614A128A1A8022E07B691B889B0852
:102040001B041A0C3B691A807B691B88BA68D31879
:10205000BB603B6902333B617B6902337B61564B5A
:102060001B8A5A00574BD2187B699A4201D8554BAC
:102070007B613B1C0E333A1C0E321288013A1A80E7
:102080003B1C0E331B88002BD7D14B4B1B8AB868E7
:10209000191C03F0E9FA031C9B081B041A0C454B9E
:1020A000DA81454B1B781B061B16172B07D0424BBA
:1020B0001B781B061B16182B01D000F05EFE414B4F
:1020C0007B610023BB603B1C0E3300221A800EE0B4
:1020D0007B691B88BA68D318BB607B6902337B615C
:1020E0003B1C0E333A1C0E32128801321A80324BDE
:1020F0001B8A3A1C0E3212889A42E9D32E4B1B8A55
:10210000B868191C03F0B0FA031C9A08BB1C1A80AB
:10211000BB1C1A88274BDA81264B5B697B612A4BF3
:102120007B603B1C0E3300221A8026E07B691B88F3
:102130009B081B041A0CBB1C1B88D31A1B041B0C0A
:102140001B041A0C7B681A807B6802337B607B69F6
:1021500002337B61184B1B8A5B001A1C194BD31886
:102160001A1C7B699A4201D8164B7B613B1C0E33CB
:102170003A1C0E32128801321A800F4B1B8A3A1C0D
:102180000E3212889A42D1D30F4B7B600C4B3B61CD
:10219000094B1B781B061B16172B03D0182B00D1DD
:1021A000F5E2F3E23B1C0E3300221A80DEE2C04669
:1021B00000080140DC1D00206404002008000240EB
:1021C000A415002078040020780C00207B680433DC
:1021D0001B881B041A0CBB1C1B88D3181B041A0C6D
:1021E0003B691A803B69023398467B681B881B0455
:1021F0001B14181CFEF710FF031C181CFEF7ECFA4A
:10220000031C0C1C181C211CF24BF14AFEF738FB76
:10221000031C0C1C1D1C261C7B6802331B881B0422
:102220001B14181CFEF7F8FE031C181CFEF7D4FA4A
:10223000031C0C1C181C211CE74AE84BFEF720FB72
:10224000031C0C1C281C311C1A1C231CFEF766F9ED
:10225000031C0C1C1D1C261C7B6804331B881B04E0
:102260001B14181CFEF7D8FE021CE14B1B68101C47
:10227000191CFEF725FF031C181CFEF7ADFA031C02
:102280000C1C281C311C1A1C231CFEF747F9031CCC
:102290000C1C1D1C261C7B6806331B881B041B148E
:1022A000181CFEF7B9FE021CD24B1B68101C191C2F
:1022B000FEF706FF031C181CFEF78EFA031C0C1C0D
:1022C000281C311C1A1C231CFEF728F9031C0C1CAB
:1022D0001D1C261C7B6808331B881B041B14181C40
:1022E000FEF79AFE031C181CFEF776FA031C0C1C62
:1022F000181C211CBA4ABB4BFEF7C2FA031C0C1C6B
:10230000281C311C1A1C231CFEF708F9031C0C1C8A
:10231000181C211CFEF74EFD031C1B041B0C1B0488
:102320001A0CBB1C1B88D3181B041B0C42461380C1
:102330003B69043398467B6802331B881B041B14DB
:10234000181CFEF769FE031C181CFEF745FA031C57
:102350000C1C181C211CA24AA24BFEF791FA031C6C
:102360000C1C1D1C261C7B6804331B881B041B14BF
:10237000181CFEF751FE021C9F4B1B68101C191CF9
:10238000FEF79EFE031C181CFEF726FA031C0C1C0D
:10239000281C311C1A1C231CFEF7C0F8031C0C1C43
:1023A0001D1C261C7B6806331B881B041B14181C71
:1023B000FEF732FE021C914B1B68101C191CFEF725
:1023C0007FFE031C181CFEF707FA031C0C1C281CBC
:1023D000311C1A1C231CFEF7A1F8031C0C1C1D1C2D
:1023E000261C7B6808331B881B041B14181CFEF773
:1023F00013FE031C181CFEF7EFF9031C0C1C181C21
:10240000211C794A794BFEF73BFA031C0C1C281C53
:10241000311C1A1C231CFEF781F8031C0C1C1D1C0C
:10242000261C7B680A331B881B041B14181CFEF730
:10243000F3FD031C181CFEF7CFF9031C0C1C181C21
:10244000211C644B624AFEF71BFA031C0C1C281C5F
:10245000311C1A1C231CFEF761F8031C0C1C181CF1
:10246000211CFEF7A7FC031C1B041B0C1B041A0CED
:10247000BB1C1B88D3181B041B0C424613803B69F2
:10248000063398467B6802331B881B041B14181CF8
:10249000FEF7C2FD031C181CFEF79EF9031C0C1C62
:1024A000181C211C4B4B4A4AFEF7EAF9031C0C1C72
:1024B0001D1C261C7B6804331B881B041B14181C62
:1024C000FEF7AAFD031C181CFEF786F9031C0C1C62
:1024D000181C211C444A454BFEF7D2F9031C0C1C66
:1024E000281C311C1A1C231CFEF718F8031C0C1C9A
:1024F0001D1C261C7B6806331B881B041B14181C20
:10250000FEF78AFD021C3D4B1B68101C191CFEF7D0
:10251000D7FD031C181CFEF75FF9031C0C1C281CBC
:10252000311C1A1C231CFDF7F9FF031C0C1C1D1C7D
:10253000261C7B6808331B881B041B14181CFEF721
:102540006BFD021C2C4B1B68101C191CFEF7B8FD00
:10255000031C181CFEF740F9031C0C1C281C311C22
:102560001A1C231CFDF7DAFF031C0C1C1D1C261C67
:102570007B680A331B881B041B14181CFEF74CFDD8
:10258000031C181CFEF728F9031C0C1C181C211C2A
:10259000104B0F4AFEF774F9031C0C1C281C311C4D
:1025A0001A1C231CFDF7BAFF031C0C1C181C211C51
:1025B000FEF700FC031C1B041B0C1B041A0CBB1CA9
:1025C0001B88D3181B041B0C424619E0C046C046AA
:1025D0000000000000000000AF946588635DB4BF98
:1025E0000E2DB29DEFA7A6BF4F232D95B723B4BFE5
:1025F000942100205C2000202C1F0020602000205F
:1026000013803B690822D21890467B6804331B88EC
:102610001B041B14181CFEF7FFFC031C181CFEF700
:10262000DBF8031C0C1C181C211C5C4B5A4AFEF7DF
:1026300027F9031C0C1C1D1C261C7B6806331B88F9
:102640001B041B14181CFEF7E7FC021C584B1B68EC
:10265000101C191CFEF734FD031C181CFEF7BCF8F7
:10266000031C0C1C281C311C1A1C231CFDF756FFD4
:10267000031C0C1C1D1C261C7B6808331B881B04B8
:102680001B14181CFEF7C8FC021C4A4B1B68101CCC
:10269000191CFEF715FD031C181CFEF79DF8031C02
:1026A0000C1C281C311C1A1C231CFDF737FF031CB3
:1026B0000C1C1D1C261C7B680A331B881B041B1466
:1026C000181CFEF7A9FC031C181CFEF785F8031C58
:1026D0000C1C181C211C324A324BFEF7D1F8031C8B
:1026E0000C1C281C311C1A1C231CFDF717FF031C93
:1026F0000C1C1D1C261C7B680C331B881B041B1424
:10270000181CFEF789FC031C181CFEF765F8031C57
:102710000C1C181C211C244A244BFEF7B1F8031C86
:102720000C1C281C311C1A1C231CFDF7F7FE031C73
:102730000C1C181C211CFEF73DFB031C1B041B0C6E
:102740001B041A0CBB1C1B88D3181B041B0C424611
:1027500013807B6804337B603B690A333B613B1C1D
:102760000E333A1C0E32128801321A80124B1B8A29
:10277000181C052102F078FF031C1B041B0C3A1CDB
:102780000E3212889A4200D220E5F6E2F5E23B1CB6
:102790000E3300221A80E0E20E2DB29DEFA7A6BFF5
:1027A000AF946588635DB4BF0000000000000000C6
:1027B0005C20002094210020640400207B68043306
:1027C0001B881B041A0CBB1C1B88D3181B041A0C77
:1027D0003B691A803B69023398467B681B881B045F
:1027E0001B14181CFEF718FC031C181CFDF7F4FF43
:1027F000031C0C1C181C211CF24BF14AFEF740F87C
:10280000031C0C1C1D1C261C7B6802331B881B042C
:102810001B14181CFEF700FC031C181CFDF7DCFF42
:10282000031C0C1C181C211CE74AE84BFEF728F877
:10283000031C0C1C281C311C1A1C231CFDF76EFEEB
:10284000031C0C1C1D1C261C7B6804331B881B04EA
:102850001B14181CFEF7E0FB021CE14B1B68101C4C
:10286000191CFEF72DFC031C181CFDF7B5FF031CFB
:102870000C1C281C311C1A1C231CFDF74FFE031CCA
:102880000C1C1D1C261C7B6806331B881B041B1498
:10289000181CFEF7C1FB021CD24B1B68101C191C34
:1028A000FEF70EFC031C181CFDF796FF031C0C1C06
:1028B000281C311C1A1C231CFDF730FE031C0C1CA9
:1028C0001D1C261C7B6808331B881B041B14181C4A
:1028D000FEF7A2FB031C181CFDF77EFF031C0C1C5B
:1028E000181C211CBA4ABB4BFDF7CAFF031C0C1C69
:1028F000281C311C1A1C231CFDF710FE031C0C1C89
:10290000181C211CFEF756FA031C1B041B0C1B048D
:102910001A0CBB1C1B88D3181B041B0C42461380CB
:102920003B69043398467B681B881B041B14181CE6
:10293000FEF772FB031C181CFDF74EFF031C0C1C5A
:10294000181C211C9F4B9E4AFDF79AFF031C0C1C70
:102950001D1C261C7B6802331B881B041B14181CBF
:10296000FEF75AFB031C181CFDF736FF031C0C1C5A
:10297000181C211C984A994BFDF782FF031C0C1C64
:10298000281C311C1A1C231CFDF7C8FD031C0C1C41
:102990001D1C261C7B6804331B881B041B14181C7D
:1029A000FEF73AFB021C904B1B68101C191CFEF72B
:1029B00087FB031C181CFDF70FFF031C0C1C281CB5
:1029C000311C1A1C231CFDF7A9FD031C0C1C1D1C2B
:1029D000261C7B6806331B881B041B14181CFEF77F
:1029E0001BFB021C814B1B68101C191CFEF768FBAB
:1029F000031C181CFDF7F0FE031C0C1C281C311CCA
:102A00001A1C231CFDF78AFD031C0C1C1D1C261C14
:102A10007B6808331B881B041B14181CFEF7FCFA88
:102A2000031C181CFDF7D8FE031C0C1C181C211CD1
:102A3000674A684BFDF724FF031C0C1C281C311C43
:102A40001A1C231CFDF76AFD031C0C1C181C211CFE
:102A5000FEF7B0F9031C1B041B0C1B041A0CBB1C57
:102A60001B88D3181B041B0C424613803B6906339A
:102A700098467B6802331B881B041B14181CFEF746
:102A8000CBFA031C181CFDF7A7FE031C0C1C181C1A
:102A9000211C4F4A4F4BFDF7F3FE031C0C1C1D1C61
:102AA000261C7B6804331B881B041B14181CFEF7B0
:102AB000B3FA021C4D4B1B68101C191CFEF700FBDF
:102AC000031C181CFDF788FE031C0C1C281C311C61
:102AD0001A1C231CFDF722FD031C0C1C1D1C261CAC
:102AE0007B6806331B881B041B14181CFEF794FA22
:102AF000021C3D4B1B68101C191CFEF7E1FA031C5D
:102B0000181CFDF769FE031C0C1C281C311C1A1C28
:102B1000231CFDF703FD031C0C1C1D1C261C7B68DD
:102B200008331B881B041B14181CFEF775FA031CC2
:102B3000181CFDF751FE031C0C1C181C211C264AF6
:102B4000264BFDF79DFE031C0C1C281C311C1A1C77
:102B5000231CFDF7E3FC031C0C1C1D1C261C7B68BE
:102B60000A331B881B041B14181CFEF755FA031CA0
:102B7000181CFDF731FE031C0C1C181C211C114BEA
:102B80000F4AFDF77DFE031C0C1C281C311C1A1C6F
:102B9000231CFDF7C3FC031C0C1C181C211CFEF796
:102BA00009F9031C1B041B0C1B041A0CBB1C1B88FF
:102BB000D3181B041B0C4246138019E0C046C046C4
:102BC00000000000000000004F232D95B723B4BF84
:102BD0000E2DB29DEFA7A6BFAF946588635DB4BF0D
:102BE000602000202C1F0020942100205C20002069
:102BF0003B690822D21890467B6802331B881B046D
:102C00001B14181CFEF708FA031C181CFDF7E4FD42
:102C1000031C0C1C181C211C784B774AFDF730FE56
:102C2000031C0C1C1D1C261C7B6804331B881B0406
:102C30001B14181CFEF7F0F9021C754B1B68101CC6
:102C4000191CFEF73DFA031C181CFDF7C5FD031CFB
:102C50000C1C281C311C1A1C231CFDF75FFC031CD8
:102C60000C1C1D1C261C7B6806331B881B041B14B4
:102C7000181CFEF7D1F9021C664B1B68101C191CAE
:102C8000FEF71EFA031C181CFDF7A6FD031C0C1C06
:102C9000281C311C1A1C231CFDF740FC031C0C1CB7
:102CA0001D1C261C7B6808331B881B041B14181C66
:102CB000FEF7B2F9031C181CFDF78EFD031C0C1C5B
:102CC000181C211C4E4A4F4BFDF7DAFD031C0C1C4F
:102CD000281C311C1A1C231CFDF720FC031C0C1C97
:102CE0001D1C261C7B680A331B881B041B14181C24
:102CF000FEF792F9031C181CFDF76EFD031C0C1C5B
:102D0000181C211C404A414BFDF7BAFD031C0C1C4A
:102D1000281C311C1A1C231CFDF700FC031C0C1C76
:102D2000181C211CFEF746F8031C1B041B0C1B047B
:102D30001A0CBB1C1B88D3181B041B0C42461380A7
:102D40007B6802337B603B690A333B613B1C0E337B
:102D50003A1C0E32128801321A802F4B1B8A181C23
:102D6000052102F081FC031C1B041B0C3A1C0E32D3
:102D700012889A4200D221E5C046284B284A9A611F
:102D8000284B1B88312B12D9264B00221A8001F0C8
:102D9000F9FD031C0BD0244B05221A80224B642220
:102DA0005A80214B04229A801F4B2222DA801B4B2F
:102DB0001B881A1C2023134017D0184B1B88042291
:102DC00013431B041A0C154B1A80144B1B8820222A
:102DD00093431B041A0C114B1A80104B5B88022280
:102DE00013431B041A0C0D4B5A80BD4606B004BC9D
:102DF0009046F0BC01BC00470E2DB29DEFA7A6BFC8
:102E00004F232D95B723B4BF000000000000000041
:102E10002C1F00206020002064040020DC1D002006
:102E2000A4150020A41D0020B802002080B500AF2A
:102E3000104B1B88082293431B041A0C0D4B1A805D
:102E40000D4B1B781B061B160D2B0FDC0A4B9B7AB8
:102E5000002B0BD1074B5A69064B9A61054B5B88D7
:102E6000042213431B041A0C024B5A80BD4680BC3B
:102E700001BC0047DC1D00206404002080B500AFC9
:102E80008023DB058022D20512881204120C012156
:102E90008A431204120C1A80BD4680BC01BC004754
:102EA00080B582B000AF021CFB1D1A70FB1D1B78A1
:102EB0001B061B160D2B02DDFB1D0D221A70FB1DC0
:102EC0001B781B061B16012B02DCFB1D02221A704D
:102ED0000E4B1B881B061A0EFB1D1B78D3181B06F6
:102EE0001B0E1B061A0E0A4B1A710A4B1B88013364
:102EF0001B041A0C074B1A80FB1D1B781B061B16A4
:102F0000181CBD4602B080BC02BC0847B8020020B5
:102F100064040020A41D002080B500AF044B1B7981
:102F20001B061B16181CBD4680BC02BC0847C046C9
:102F30006404002080B582B000AF021CFB1D1A7033
:102F4000FB1D1B781B061B16022B02DDFB1D02223C
:102F50001A70FB1D1B787F2B02D9FB1D00221A70F3
:102F60000A4BFA1D12785A71094B1B8801331B0456
:102F70001A0C074B1A80054B5B791B061B16181C95
:102F8000BD4602B080BC02BC0847C04664040020B5
:102F9000A41D002080B500AF044B5B791B061B16F7
:102FA000181CBD4680BC02BC0847C0466404002013
:102FB00080B582B000AF021CBB1D1A80BB1D002172
:102FC0005A5E134B9A4202DABB1D114A1A80BB1D8E
:102FD00000215A5EFA235B009A4203DDBB1DFA22F0
:102FE00052001A800B4B5A88BB1D1B88D3181B0438
:102FF0001B0C1B041A0C084BDA80BB1D1B881B041E
:103000001B14181CBD4602B080BC02BC0847C04659
:103010000CFEFFFFB80200206404002080B500AF62
:10302000044BDB881B041B14181CBD4680BC02BC6F
:103030000847C0466404002080B582B000AF021C7F
:10304000FB1D1A70FB1D1B781B061B16002B02DCD8
:10305000FB1D01221A70FB1D1B781B061B16182B6B
:1030600002DDFB1D18221A700B4B9B881B061A0EE3
:10307000FB1D1B78D3181B061B0E1B061A0E074BD5
:103080001A70FB1D1B781B061B16181CBD4602B0D0
:1030900080BC02BC0847C046B8020020640400207F
:1030A00080B500AF044B1B781B061B16181CBD46D1
:1030B00080BC02BC0847C0466404002080B582B0D2
:1030C00000AF021CBB1D1A80BB1D00215B5E002BE4
:1030D00002DABB1D00221A80BB1D00215A5E0E4B76
:1030E0001B8A2E3BFF3B9A4207DD0B4B1B8A2E3B74
:1030F000FF3B1B041A0CBB1D1A80074BBA1D12881C
:103100005A80054B5B881B041B14181CBD4602B07B
:1031100080BC02BC0847C0466404002080B500AFF4
:10312000044B5B881B041B14181CBD4680BC02BCEE
:103130000847C0466404002080B582B000AF021C7E
:10314000FB1D1A70FB1D1B787F2B02D9FB1D002273
:103150001A70FB1D1B781B061B16022B02DDFB1DC4
:1031600002221A700A4BFA1D12789A72094B1B88B8
:1031700001331B041A0C074B1A80054B9B7A1B0664
:103180001B16181CBD4602B080BC02BC0847C046D6
:1031900064040020A41D002080B500AF044B9B7A7E
:1031A0001B061B16181CBD4680BC02BC0847C04647
:1031B0006404002080B582B000AF021CFB1D1A70B1
:1031C000FB1D1B787F2B02D9FB1D00221A70FB1DF3
:1031D0001B781B061B16012B02DDFB1D01221A703A
:1031E000124BFA1D1278DA72114B1B881D2B12D963
:1031F0000F4B00221A8001F0C5FB031C0BD00D4BB6
:1032000024221A800B4B64225A800A4B07229A8090
:10321000084B2222DA80054BDB7A1B061B16181C92
:10322000BD4602B080BC02BC0847C0466404002012
:10323000A41D0020B802002080B500AF044BDB7A4B
:103240001B061B16181CBD4680BC02BC0847C046A6
:103250006404002080B582B000AF021CBB1D1A8040
:10326000BB1D00215A5E134B9A4202DABB1D114A64
:103270001A80BB1D00215A5E9623DB009A4203DDB3
:10328000BB1D9622D2001A800B4BDA88BB1D1B880F
:10329000D3181B041B0C1B041A0C084B9A81BB1D72
:1032A0001B881B041B14181CBD4602B080BC02BC4A
:1032B0000847C04650FBFFFFB8020020640400200E
:1032C00080B500AF044B9B891B041B14181CBD4622
:1032D00080BC02BC0847C0466404002080B582B0B0
:1032E00000AF021CBB1D1A80BB1D1A880E4B9A42F0
:1032F00003D8BB1D802292001A80BB1D1A88802330
:10330000DB009A4203D9BB1D8022D2001A80074BF2
:10331000BA1D12881A82054B1B8A181CBD4602B0C2
:1033200080BC02BC0847C046FF01000064040020C6
:1033300080B500AF034B1B8A181CBD4680BC02BC85
:103340000847C0466404002080B582B000AF021C6C
:10335000FB1D1A70FB1D1B78062B02D9FB1D0622D4
:103360001A70094BFA1D12781A71084B1B88013329
:103370001B041A0C054B1A80034B1B79181CBD4605
:1033800002B080BC02BC0847DC1D0020A41D002048
:1033900080B500AF034B1B79181CBD4680BC02BC36
:1033A0000847C046DC1D002080B500AF034B1B88DA
:1033B000181CBD4680BC02BC0847C046DC1D00206E
:1033C00080B500AF114B1B88042213431B041A0C59
:1033D0000E4B1A800E4B1B88272B12D90C4B002248
:1033E0001A8001F0CFFA031C0BD00A4B05221A8079
:1033F000084B36225A80074B15229A80054B222211
:10340000DA80BD4680BC01BC0047C046DC1D002000
:10341000A41D0020B802002080B500AF094B1B8816
:10342000042293431B041A0C064B1A80064B1B887C
:1034300001331B041A0C044B1A80BD4680BC01BC2E
:103440000047C046DC1D0020A41D002080B500AF51
:10345000044BDB891B041B14181CBD4680BC02BC3A
:103460000847C046DC1D002080B582B000AF021CBA
:10347000BB1D1A80BB1D00215A5E0F4B9A4202DA17
:10348000BB1D0D4A1A80BB1D00215A5EFA235B004A
:103490009A4203DDBB1DFA2252001A80074BBA1D67
:1034A00012881A81BB1D1B881B041B14181CBD46E7
:1034B00002B080BC02BC08470CFEFFFF6404002081
:1034C00080B500AF044B1B891B041B14181CBD46A0
:1034D00080BC02BC0847C0466404002080B582B0AE
:1034E00000AF021CBB1D1A80064B5A88BB1D1B88EF
:1034F00013431B041A0C034B5A80BD4602B080BC18
:1035000001BC0047DC1D002080B582B000AF021C6A
:10351000BB1D1A800A4B5B881B041B0CBA1D12884A
:10352000D2431204120C13401B041B0C1B041A0C74
:10353000034B5A80BD4602B080BC01BC0047C04668
:10354000DC1D002080B500AFBD4680BC01BC00473B
:1035500080B582B000AF021CBB1D1A8008E0BB1D05
:103560001B881B041B0C013B1B041A0CBB1D1A807F
:10357000BB1D1B881B041B0CF1D1BD4602B080BCD7
:1035800001BC0047B0B584B002AFD44B5B881A1CB5
:103590000823134009D0D14B5B88082293431B04B6
:1035A0001A0CCE4B5A8003F06DFFCC4B5B881A1C73
:1035B000012313400BD0C94B5B88012293431B04AA
:1035C0001A0CC64B5A8003F05DFF00F06BFAC34B38
:1035D0005B881A1C0223134000D11AE2BF4B5B88A0
:1035E000022293431B041A0CBC4B5A80A0235B009D
:1035F000002200920020DA211A1C162303F02CFF6F
:10360000B74B1B791B061B169A1E131C9B009B189D
:10361000B44A9A18B44B00210091B449019110208A
:10362000E12103F03FFFAE4B5B791B061B169A00AE
:10363000AF4BD218AC4B00210091AC4901913C201A
:10364000E12103F02FFFA64B1B781B061B165A1E09
:10365000131C5B009B185B00A64A9A18FC23DB0036
:1036600000210091A14901917320E12103F01AFF8B
:103670009B4B9B7A1B061A16131C9B009B189E4A99
:103680009A189E4B0021009198490191C320E12195
:1036900003F008FF924BDB7A1B061A0E82235900B7
:1036A000964B0020009096480190081CE32103F0FF
:1036B0004BFF8A4B1B79032B2CD87B1D874A127931
:1036C0001A707B1D1A788F4BD200D05A7B1D1A7846
:1036D0008C490223D2008A18D31819887B1D1A78C6
:1036E000884C0423D200A218D3181A887B1D1C789A
:1036F000844D0623E4002C19E3181B8800040014F1
:1037000009040914120412141B041B147E4C0094A7
:10371000FDF7BEFE7D4B00220092744A01920E20FE
:1037200000211A1C002303F0BDFE6C4B1B881A1CE1
:10373000042313400BD0764B002200926B4A019277
:103740000E2000211A1C1F2303F0ACFE0AE0714A70
:10375000FC23DB0000210091644901910E2000212F
:1037600003F0A0FE5D4B1B891B041B0C033B1B04D9
:103770001B0C00220092684A01920220191C0122AF
:10378000002303F0E1FE564BDB881B041B0C752263
:10379000D31A1B041A0CBB1D1A80BB1D00229B5E92
:1037A000102B02DCBB1D11221A80BB1D00229B5E68
:1037B000D92B02DDBB1DD9221A80484B1B79062B61
:1037C00001D1514B00E0484BBA1C1380BB1D1B8834
:1037D000033B1B041A0CBB1C1B88002100914E49A3
:1037E00001910220111C012203F0AEFE3B4BBA1DD9
:1037F00012881A81394BDA88384B5B79120412141B
:103800001B041B1400210091101C08211A1C052305
:1038100003F022FEFC23DB0000936B200621012233
:10382000082303F019FEFC23DB0000936B20062124
:103830000422012303F010FEFC23DB0000936B2025
:103840000E210422012303F007FEFC23DB0000937A
:10385000D52006210122082303F0FEFDFC23DB0016
:103860000093D22006210422012303F0F5FDFC235E
:10387000DB000093D2200E210422012303F0ECFD93
:10388000FC23DB0000936E200A216522012303F054
:10389000E3FD134B5B881B041B14652253431A1C66
:1038A0000F4B1B8A101C191C01F0DEFE031C1B06AB
:1038B0001A0E7B1D6E321A70094B1B8A1748191C91
:1038C00001F0D2FE031C1B041A0C7B1C1A70034B64
:1038D0001B79052B24D10C4B24E0C046DC1D0020B5
:1038E000640400201CA10008FF070000040200205F
:1038F00088A1000894A100082CA200085FB3000072
:1039000030010020FCA00008E0FF00005CA20008DD
:1039100068A2000870A20008100100205C76000078
:10392000FC23DB00BA1C13807B1D1B781B041A0CC4
:103930007B1C1B781B041B0C120412141B041B148D
:10394000B91C09880091101C08211A1C052303F0DA
:1039500083FD7B1D1B781B041A0C494BDA80484BF6
:103960007A1C12785A71464B5B891B041B0C033B73
:103970001B041B0C434A0021009143490191101C78
:10398000191C0222002303F0DFFD404B9B891B041E
:103990001B149B101B041B0C1B041A0C3B4BDB88D9
:1039A0001B041B0CD3181B041B0C7522D31A1B04FD
:1039B0001A0CBB1D1A80BB1D00229B5E102B02DC63
:1039C000BB1D11221A80BB1D00229B5ED92B02DD7C
:1039D000BB1DD9221A802A4B1B79042B01D12C4BF9
:1039E00000E02C4BBA1C1380BB1D1B88033B1B043F
:1039F0001A0C2449BB1C1B8800200090224801900F
:103A0000081C111C022203F09FFD1D4BBA1D1288D9
:103A10005A811B4B5B881A1C102313401AD0184B79
:103A20005B88102293431B041A0C154B5A80144BCD
:103A30001B7FDA00184BD218114B1B7F191C174B38
:103A40004900CB5A0021009115490191F020002135
:103A500003F028FD0A4B5B881A1C0423134009D08D
:103A6000074B5B88042293431B041A0C044B5A80B7
:103A700000F0EAF8BD4602B0B0BC01BC0047C04649
:103A8000DC1D00203701000010010020640400202C
:103A9000E0FF00005FB300003CA2000854A2000851
:103AA0000402002080B584B002AFFB1D01221A7011
:103AB00021E0FB1D1B781B041B0C1A1C9200D31861
:103AC0001A1C91001A1C0B1CD3181B041B0C0A3364
:103AD0001B041B0C1B041B0C1B041B14584A0092D8
:103AE000181C11210122C82303F0B6FCFB1DFA1D8E
:103AF000127801321A70FB1D1B780B2BD9D9FB1DD4
:103B000001221A7022E0FB1D1B781B041B0C1A1CDF
:103B10009200D3181A1C91001A1C0B1CD3181B04FA
:103B20001B0C11331B041B0C1B041B0C1B041B1450
:103B300096225200424900910A20191C012303F0E9
:103B40008BFCFB1DFA1D127801321A70FB1D1B78CD
:103B5000072BD8D996235B003A4A00920A201121FC
:103B60001A1C012303F078FC96235B00354A00926F
:103B70000A20D9211A1C012303F06EFC314B00935B
:103B80000A2011210122C82303F066FC9B235B005D
:103B90002C4A0092181C11210122C82303F05CFC5E
:103BA000FB1D01221A701CE0FB1D1B781B041B0C63
:103BB0001A1C9200D3181B041B0C0A331B041B0C89
:103BC0001B041B0C1B041B141D4A0092181C7321A0
:103BD0000122052303F040FCFB1DFA1D127801327F
:103BE0001A70FB1D1B783B2BDED9FB1D01221A70BE
:103BF0001CE0FB1D1B781B041B0C1A1C9200D31825
:103C00001B041B0C11331B041B0C1B041B0C1B047F
:103C10001B140B4A00929E20191C0522012303F05D
:103C20001BFCFB1DFA1D127801321A70FB1D1B785C
:103C3000272BDED9BD4602B080BC01BC0047C04680
:103C4000CB5A0000FBDE000090B589B000AF7D4B81
:103C50001B881A1C4023134004D07B4B7B617B4B99
:103C60003B6103E07A4B7B617A4B3B61754B9A6910
:103C7000794B5B881B041B145B00D318FB60764BED
:103C80001B8A5A00754BD218FB689A4206D8724BB1
:103C90001B8A5B005B42FA68D318FB606E4BDB88C3
:103CA0001B041A0C6C4B1B891B041B0CD31A1B0422
:103CB0001A0C3B1C0A331A80FB681A883B1C0A3317
:103CC0001B88D3181B041A0C3B1C1A331A803B1C8C
:103CD0001A3300215A5E624B9A4203DD3B1C1A33B1
:103CE0005F4A1A803B1C1A3300215A5E5D4B9A4290
:103CF00004DC3B1C1A33CE2252001A803B1C1E33BC
:103D00000B221A8081E0FB681A883B1C1C331A8046
:103D10003B1C1C331A883B1C0A331B88D3181B041A
:103D20001A0C3B1C1C331A803B1C1C3300215A5EAE
:103D30004B4B9A4203DD3B1C1C33494A1A803B1C07
:103D40001C3300215A5E474B9A4204DC3B1C1C3357
:103D5000CE2252001A803C1C08343B1C1C3300212C
:103D60005A5E3B1C1A3300215B5E101C191CFDF7C8
:103D700043FE031C2380BC1D3B1C1C3300215A5EE8
:103D80003B1C1A3300215B5E101C191CFDF752FE10
:103D9000031C23803B1C1A333A1C1C3212881A80E5
:103DA000BB1D1B881B061B0E7522D31A1B061A0E81
:103DB0007B691A707B6901337B61BB1D1B881B0605
:103DC0001A0E3B1C08331B881B061B0ED31A1B063E
:103DD0001B0E01331B061A0E3B691A703B69013337
:103DE0003B61FB680233FB601B4B1B8A5A001B4B79
:103DF000D218FB689A4201D8184BFB603B1C1E335B
:103E00003A1C1E32128801321A803B1C1E331A885B
:103E1000154B9A4200D876E7002000F029F8FFF70A
:103E200041FE084B1B88402253401B041A0C054BD3
:103E30001A800E4B181C00F01BF8BD4609B090BC50
:103E400001BC0047DC1D0020301F0020781400203A
:103E500064200020001E002064040020A41500201F
:103E6000630200009B01000035010000FF07000015
:103E700080B588B002AF021CBB1D1A80374B1B886F
:103E80001A1C4023134032D0354B3B61354BFB604D
:103E90003B1C16330B221A8022E03B1C1633198878
:103EA0003B691B781A1C3B6901333B61FB681B783B
:103EB000F8680130F86009040914120412141B0494
:103EC0001B14B81D00880090081C111C012203F06F
:103ED000C3FA3B1C16333A1C1632128801321A8080
:103EE0003B1C16331A88204B9A42D6D931E01F4B1F
:103EF0003B611F4BFB603B1C16330B221A8022E0F8
:103F00003B1C163319883B691B781A1C3B6901332B
:103F10003B61FB681B78F8680130F86009040914FC
:103F2000120412141B041B14B81D00880090081CF6
:103F3000111C012203F090FA3B1C16333A1C163276
:103F4000128801321A803B1C16331A88064B9A429B
:103F5000D6D9BD4606B080BC01BC0047DC1D0020A0
:103F600064200020001E002035010000301F0020CA
:103F70007814002080B500AF564B1B8A1B041B0C25
:103F80001A1C0223134068D0524B9B8E1B041A0C40
:103F9000514B1A824F4B4F4A92891204120C022144
:103FA0008A431204120C9A814A4B4A4A128C120418
:103FB000120C01218A431204120C1A84454B464A02
:103FC000118A464A108A454AD2891204120C821A72
:103FD0001204120C8A181204120C1A873D4B3D4A27
:103FE000128A1204120C04218A431204120C1A823F
:103FF0003A4B1B781B061B160D2B03DC374B9B7AA9
:10400000002B09D0334B334A92891204120C04213D
:104010000A431204120C9A812F4B1B88022213436D
:104020001B041A0C2C4B1A802A4B2A4A128A12049F
:10403000120C02218A431204120C1A82264B02220D
:104040001A77254B5B88102213431B041A0C224B52
:104050005A80234B802212025A611E4B1B8A1B047A
:104060001B0C1A1C042313402FD01E4B1D4A126830
:1040700001218A431A60174B164A128A1204120C45
:1040800004218A431204120C1A82124B114A92899B
:104090001204120C04218A431204120C9A81802308
:1040A000DB058022D20512881204120C01218A43FA
:1040B0001204120C1A80FDF751FF074B1B880122D6
:1040C00013431B041A0C044B1A80BD4680BC01BC70
:1040D0000047C046002C0140DC1D00206404002085
:1040E000000801400800024080B582B000AF204BBC
:1040F0001A680223134035D01D4B1D4A1268022155
:104100008A431A601A4BDA6CBB1D1A80194B5B6923
:10411000BA1D128892081204120C1A80154B5A69A3
:10412000154B1A60134B5B699A1C124B5A61114B69
:104130005A69124BD968124B1B8A5B00CB189A4202
:1041400008D30C4B5A690E4B1B8A5B005B42D2189A
:10415000084B5A61074B1B88082213431B041A0C97
:10416000044B1A80BD4602B080BC01BC0047C0466B
:1041700000240140DC1D0020FC1D0020080002403E
:104180006404002080B500AF244B1A68022313405A
:1041900005D0224B214A526802210A435A601F4B24
:1041A0001A680423134034D01D4B1D4A128A12048E
:1041B000110C1C4A0A401204120C1A82174B174A9F
:1041C000526804210A435A60174B174A12680421A7
:1041D0008A431A60124B124A92891204120C02216D
:1041E0000A431204120C9A810D4B0D4A128C1204D0
:1041F000120C01210A431204120C1A840B4B0122E7
:104200001A770A4B5B88102213431B041A0C074BC6
:104210005A80BD4680BC01BC0047C0460000024039
:10422000002C0140FDFDFFFF08000240DC1D0020C6
:1042300080B582B000AFFB1D08221A7008E0094B60
:10424000181CFFF785F9FB1DFA1D1278013A1A7048
:10425000FB1D1B78002BF2D1BD4602B080BC01BC17
:104260000047C046DCFF000080B588B000AFB960F1
:104270007A603B1C0F33021C1A703B1C1C3300225B
:104280001A803B1C1833394A1A803B1C1F3300220A
:104290001A704CE03B1C1B3301221A703BE03B1CA4
:1042A0001F331B78BA68D3181B783A1C1B3212785C
:1042B00013401B061B0E5A1E93411B061A0E3B1C75
:1042C00017331A703B1C1C331B88DB0B1B041A0CA6
:1042D0003B1C16331A703B1C1C333A1C1C321288D0
:1042E00052001A803A1C17323B1C163312781B7886
:1042F0009A4209D03B1C1C33391C1C313A1C183221
:10430000098812884A401A803B1C1B333A1C1B3216
:10431000127852001A703B1C1B331B78002BBED145
:104320003B1C1F333A1C1F32127801321A703A1CA0
:104330001F323B1C0F3312781B789A42AAD33B1CC6
:104340001C331B881B061A0E7B681A707B680133AE
:104350003A1C1C321288120A1204120C1206120E97
:104360001A70BD4608B080BC01BC00470580FFFF45
:1043700080B500AF02F0A0FE0E4B802212015A6100
:104380000C4B8022D2005A610B4B181CFFF7E0F84F
:10439000084B802212011A61084B181CFFF7D8F84D
:1043A000064B181CFFF7D4F802F07AFEBD4680BC1D
:1043B00001BC0047000C014060EA0000DCFF000087
:1043C00080B582B000AF78600A1CFB1C1A7002F046
:1043D0001DFDC82002F06EFD02F0D2FD031C03D1CA
:1043E00002F03EFD002326E0032002F063FD02F010
:1043F000C7FD031C18D102F033FD00231BE07B68CE
:104400001B787A6801327A60181C02F053FD02F0C2
:10441000B7FD031C03D102F023FD00230BE0FB1CBE
:10442000FA1C1278013A1A70FB1C1B78002BE6D19B
:1044300002F016FD0123181CBD4602B080BC02BC70
:104440000847C04680B584B000AF786002F0DEFC5B
:10445000C92002F02FFD02F093FD031C03D102F0EE
:10446000FFFC00233EE002F065FD021C3B1C0F3305
:104470001A7002F09FFD7B683A1C0F3212781A7096
:104480007B6801337B603B1C0F333A1C0F32127880
:10449000023A1A7012E002F04DFD031C1B061A0EC0
:1044A0007B681A707B6801337B6002F083FD3B1CE4
:1044B0000F333A1C0F321278013A1A703B1C0F333B
:1044C0001B78002BE7D102F035FD031C1B061A0EEA
:1044D0007B681A707B6801337B6002F093FD02F009
:1044E000BFFC0123181CBD4604B080BC02BC0847B9
:1044F00080B500AF02F08AFCC82002F0DBFC02F0BD
:104500003FFD022002F0D6FC02F03AFD02F0A8FCCA
:10451000BD4680BC01BC004780B500AF02F076FC10
:10452000C82002F0C7FC02F02BFD002002F0C2FC04
:1045300002F026FD02F094FCBD4680BC01BC0047A1
:1045400080B59CB000AF3B60FB1D1870BB1D19709F
:104550003B1D1A803B1C78331B7807331B061A0E51
:104560003B1C08331A703B1C0833FA1D12785A7032
:104570003B1C0833BA1D12789A703B1C0833033376
:104580003A1D12881A803B1C6F3300221A7012E009
:104590003B1C6F331B7805333A6811783A1C08329C
:1045A000D1543B6801333B603B1C6F333A1C6F3284
:1045B000127801321A703A1C6F323B1C7833127831
:1045C0001B789A42E4D33B1C78331B7805331B06D7
:1045D000190E3B1C78331B7805333A1C0832D3186C
:1045E0003A1C0832081C111C1A1CFFF73DFE3B1C2C
:1045F00078331B7807331B061B0E3A1C0832101C3D
:10460000191CFFF7DDFE181CBD461CB080BC02BCA7
:104610000847C04680B5B0B002AF3A60FB1D021C2F
:104620001A70BB1D0A1C1A70FFF7A2FE02F012FDE1
:10463000FFF772FFBC4B14220092162000210022CB
:10464000FFF77EFFFFF7F4FD3B1C2C33181CFFF730
:10465000F9FE031C01D180238DE13B1C2C331B7818
:10466000232B01D0812386E13B1CB63300221A8024
:1046700013E03B1CB6331B883A1CB6321288013259
:10468000391C2C31895C3A1C5032D1543B1CB63356
:104690003A1CB632128801321A803B1CB6331B8892
:1046A0001F2BE6D9BB1D1B781B041B0C002200929C
:1046B000152002211A1C0023FFF742FFFFF7B8FD67
:1046C0003B1C2C33181CFFF7BDFE031C01D18223B9
:1046D00051E13B1C2C335B78002B01D083234AE152
:1046E000FB1D1B781B041B0CDB001B041B0C002296
:1046F0000092022082211A1C0023FFF721FFFFF7FE
:1047000097FD3B1C0833181CFFF79CFE031C01D1CE
:10471000842330E13B1C08331B78232B14D08523E2
:1047200029E13B1CB6331B883A1CB6321288203A6A
:104730007D49895C3A1C5032D1543B1CB6333A1C3B
:10474000B632128801321A803B1CB6331B88332BD9
:10475000E7D93B1CB6331B883A1C50321621D15482
:104760003B1CB6333A1CB632128801321A803B1C0D
:10477000B6331B883A1C50320021D1543B1CB6334F
:104780003A1CB632128801321A803B1CB6331B88A1
:104790003A1C50320021D1543B1CB6333A1CB6327D
:1047A000128801321A803A1C50323B1C2C33101CE8
:1047B00037211A1C00F0D6FA3B1CB63300221A80AF
:1047C00011E03B1CB6331B883A1CB632128857499D
:1047D000895C3A1C5032D1543B1CB6333A1CB63279
:1047E000128801321A803B1CB6331B881F2BE8D974
:1047F0003B1CB6331B883A1C50321521D1543B1C4C
:10480000B6333A1CB632128801321A803B1CB633DA
:104810001B883A1C50320221D1543B1CB6333A1C3F
:10482000B632128801321A803B1CB6331B883A1C00
:104830005032D31805221A803B1CB6333A1CB632CC
:10484000128802321A803B1CB6331B883A1C503245
:10485000EE21D1543B1CB6333A1CB63212880132D9
:104860001A803B1CB6331B883A1C50320121D154AC
:104870003B1CB6333A1CB632128801321A803B1CFC
:10488000B6331B883A1C50322321D1543B1CB6331B
:104890003A1CB632128801321A800DE03B1CB63346
:1048A0001B883A1C50320021D1543B1CB6333A1CB1
:1048B000B632128801321A803B1CB6331B883F2B5C
:1048C000ECD913E03B1CB6331B883A1CB632128875
:1048D000403A391C2C31895C3A1C5032D1543B1C73
:1048E000B6333A1CB632128801321A803B1CB633FA
:1048F0001B885F2BE6D93A1C50323B1C2C33101C12
:1049000060211A1C00F02EFA021C3B1CB6331A80E0
:104910003B1CB6331B88002B01D086232BE03B1CAD
:10492000B63300221A8020E0BC0100203C010020A8
:104930003B1CB6331B883A68D3183A1CB63212882F
:104940000132391C0831895C3A1CB6321288381C95
:104950002C30825C4A401206120E1A703B1CB63391
:104960003A1CB632128801321A803B1CB6331B88BF
:104970001F2BDDD90023181CBD462EB080BC02BC05
:104980000847C04680B5AEB002AFFFF7F1FC02F0B9
:1049900061FBFFF7C1FDD14B1422009216200021CC
:1049A0000022FFF7CDFDFFF743FC3B1C2433181C0E
:1049B000FFF748FD031C00D185E13B1C24331B7825
:1049C000232B00D081E13B1CAE3300221A8013E080
:1049D0003B1CAE331B883A1CAE3212880132391CA4
:1049E0002431895C3A1C4832D1543B1CAE333A1C0A
:1049F000AE32128801321A803B1CAE331B881F2B4B
:104A0000E6D9002300931520022105220023FFF799
:104A100097FDFFF70DFC3B1C2433181CFFF712FD1C
:104A2000031C00D153E13B1C24335B78002B00D0E6
:104A30004FE1002300930220822140220023FFF750
:104A40007FFDFFF7F5FB3B1C181CFFF7FBFC031C6D
:104A500000D140E13B1C1B78232B13D043E13B1CCE
:104A6000AE331B883A1CAE321288203A9B49895CCF
:104A70003A1C4832D1543B1CAE333A1CAE32128839
:104A800001321A803B1CAE331B88332BE7D93B1C09
:104A9000AE331B883A1C48321621D1543B1CAE332E
:104AA0003A1CAE32128801321A803B1CAE331B888E
:104AB0003A1C48320021D1543B1CAE333A1CAE3272
:104AC000128801321A803B1CAE331B883A1C4832D4
:104AD0000021D1543B1CAE333A1CAE321288013255
:104AE0001A803A1C48323B1C2433101C37211A1CF4
:104AF00000F038F93B1CAE3300221A8011E03B1C59
:104B0000AE331B883A1CAE3212887549895C3A1C58
:104B10004832D1543B1CAE333A1CAE3212880132BB
:104B20001A803B1CAE331B881F2BE8D93B1CAE33CD
:104B30001B883A1C48321521D1543B1CAE333A1C19
:104B4000AE32128801321A803B1CAE331B883A1CED
:104B500048320221D1543B1CAE333A1CAE3212888B
:104B600001321A803B1CAE331B883A1C4832D318E2
:104B700005221A803B1CAE333A1CAE321288023238
:104B80001A803B1CAE331B883A1C4832EE21D154AC
:104B90003B1CAE333A1CAE32128801321A803B1CE9
:104BA000AE331B883A1C48320121D1543B1CAE3332
:104BB0003A1CAE32128801321A803B1CAE331B887D
:104BC0003A1C48322321D1543B1CAE333A1CAE323E
:104BD000128801321A800DE03B1CAE331B883A1C50
:104BE00048320021D1543B1CAE333A1CAE321288FD
:104BF00001321A803B1CAE331B883F2BECD913E0EB
:104C00003B1CAE331B883A1CAE321288403A391C2A
:104C10002431895C3A1C4832D1543B1CAE333A1CD7
:104C2000AE32128801321A803B1CAE331B885F2BD8
:104C3000E6D93A1C48323B1C2433101C60211A1C54
:104C400000F090F8021C3B1CAE331A803B1CAE33C4
:104C50001B88002B46D13B1CAE3300221A801BE080
:104C60003B1CAE331B883A1CAE3212880132391C11
:104C7000895C3A1CAE321288381C2430825C4A406F
:104C80001206110E3A1C4832D1543B1CAE333A1C6A
:104C9000AE32128801321A803B1CAE331B881F2BA8
:104CA000DED93A1C48323B1C2020111C1A1CFFF78D
:104CB000DBFA3B1C1B781A1C3B1C5B78D318DD2BE2
:104CC00011D1002310E0C0460DE0C0460BE0C04605
:104CD00009E0C04607E0C04605E0C046BC01002030
:104CE0003C010020C0460123181CBD462CB080BCEE
:104CF00002BC084780B582B000AF78607B68181CA2
:104D000000F05EFB0023181CBD4602B080BC02BC54
:104D10000847C04680B584B000AFF860B9607A60DB
:104D2000F968BA687B68081C111C1A1C00F06CFB3F
:104D30000023181CBD4604B080BC02BC0847C04616
:104D400080B582B000AF786039607A683B68101C2B
:104D5000191C00F0BFFB0023181CBD4602B080BC2C
:104D600002BC084780B5B6B000AFF860B9607A60A1
:104D70003B1C1433181CFFF7BDFF031CD422D219AF
:104D80001360D422D2191368002B03D0D422D21975
:104D900013682AE0391C1431FA68BB68081C111C1E
:104DA0001A1CFFF7B7FF031CD422D2191360D422B8
:104DB000D2191368002B03D0D422D219136814E03F
:104DC0003A1C14327B68101C191CFFF7B9FF031C36
:104DD000D422D2191360D422D2191368002B03D025
:104DE000D422D219136800E00023181CBD4636B047
:104DF00080BC02BC0847C04680B5D8B000AFF860A0
:104E0000B9607A600023AE204000C019036000231F
:104E1000AC214900C9190B600023AC225200D21901
:104E20001360B9E2AC204000C01903689B01BA6866
:104E3000D318A8214900C9190B600023AE225200E3
:104E4000D21913605FE0AE204000C019036803333D
:104E5000AE214900C9190A68A8204000C01901689C
:104E60008A1811788E4AB0204000C0198218D15497
:104E7000AE214900C9190B680233AE204000C019A9
:104E800002680132A8204000C01901688A18117810
:104E9000834AB0204000C0198218D154AE21490085
:104EA000C9190B680133AE204000C01902680232F4
:104EB000A8204000C01901688A181178784AB020EB
:104EC0004000C0198218D154AE214900C9190B689D
:104ED0000333A8204000C0190268D3181A78704B19
:104EE000B0204000C019C118AE204000C0190368AE
:104EF000CB181A70AE214900C9190B680433AE22D1
:104F00005200D2191360AE204000C01903683F2B35
:104F100099DD1023AA214900C9190B608AE0AA2251
:104F20005200D21913681A1C0F3A5D4BB020400092
:104F3000C019C3189200D358A6214900C9190B60A3
:104F4000A6235B00DB191A680723DA41A62040007C
:104F5000C01901681223081CD841031C5A40A6211D
:104F60004900C9190B68DB085340A4225200D2192A
:104F70001360AA204000C01903689A1E484BB02154
:104F80004900C919CB189200D358A6225200D21951
:104F90001360A6235B00DB191A681123DA41A620EF
:104FA0004000C01901681323081CD841031C5A4053
:104FB000A6214900C9190B689B0A5340A22252003E
:104FC000D2191360AA204000C01903681A1C103AB5
:104FD000334BB0214900C919CB189200D258A420F4
:104FE0004000C0190368D218AA214900C9190B68EA
:104FF000D91F2B4BB0204000C019C3188900CB58D3
:10500000D218A2214900C9190B68D118244BB0222B
:105010005200D219D318AA204000C0190268920089
:10502000D150AA214900C9190B680133AA225200A4
:10503000D2191360AA204000C01903683F2B00D882
:105040006DE70023AE214900C9190B601BE0FB6826
:10505000AE204000C019026822329200D158114B94
:10506000B0225200D219D318AE204000C0190268F5
:105070009200D150AE214900C9190B680133AE220C
:105080005200D2191360AE204000C0190368072BEC
:10509000DDDD0023AE214900C9190B603BE1C046AC
:1050A000D4FEFFFFB4FEFFFFC24BB0225200D21964
:1050B000D3181A680223DA41BE4BB0204000C01951
:1050C000C31819680D23081CD841031C5A40B94B5A
:1050D000B0214900C919CB1819681623081CD841FA
:1050E000031C5340A4214900C9190B60B14BB022E5
:1050F0005200D219D3181A68AE4BB0204000C01924
:10510000C3185B681A40AB4BB0214900C919CB18D2
:105110001968A84BB0204000C019C3189B680B4009
:105120005A40A44BB0214900C919CB185968A14B6A
:10513000B0204000C019C3189B680B405340A02109
:105140004900C9190B60A4235B00DB191A68A02071
:105150004000C0190368D3189E214900C9190B608B
:10516000944BB0225200D219D3181A690623DA419F
:10517000904BB0204000C019C31819690B23081CBC
:10518000D841031C5A408B4BB0214900C919CB1898
:1051900019691923081CD841031C5340A221490056
:1051A000C9190B60834BB0225200D219D3181A6967
:1051B000804BB0204000C019C3185B691A407D4B7A
:1051C000B0214900C919CB181B69D943794BB020CC
:1051D0004000C019C3189B690B4053409C214900F3
:1051E000C9190B60734BB0225200D219D318DA6977
:1051F000A2204000C0190368D2189C214900C91997
:105200000B68D2186C4BAE204000C01901688900B1
:10521000CB58D218694BB0214900C919CB18AE2020
:105220004000C01901688900CB58D3189A21490061
:10523000C9190B605F4BB0225200D219D3189A697A
:105240005C4BB0204000C019C318DA61594BB02143
:105250004900C919CB185A69564BB0204000C019F3
:10526000C3189A61534BB0214900C919CB181A6968
:10527000504BB0204000C019C3185A614D4BB021AB
:105280004900C919CB18DA689A204000C019036890
:10529000D218484BB0214900C919CB181A61454BA7
:1052A000B0225200D219D3189A68424BB020400065
:1052B000C019C318DA603F4BB0214900C919CB1897
:1052C0005A683C4BB0204000C019C3189A60394B53
:1052D000B0214900C919CB181A68364BB0204000DC
:1052E000C019C3185A609A214900C9190A689E203A
:1052F0004000C0190368D2182E4BB0214900C919CB
:10530000CB181A60AE225200D21913680133AE20B6
:105310004000C0190360AE214900C9190B683F2B3A
:1053200000DCC1E60023AE225200D219136024E053
:10533000FB68AE204000C019026822329200D258A9
:105340001C4BB0214900C919CB18AE204000C01930
:1053500001688900CB58D118FB68AE204000C01905
:10536000026822329200D150AE214900C9190B685F
:105370000133AE225200D2191360AE204000C01992
:105380000368072BD4DDAC214900C9190B68013330
:10539000AC225200D2191360AC235B00DB191A68EF
:1053A0007B689A4200D23DE5BD4658B080BC01BC46
:1053B0000047C046B4FEFFFF98A20008D4FEFFFFDE
:1053C00080B584B000AF78607B68181C0021A822EB
:1053D00000F042FB0023FB600BE00A4BFA689200EE
:1053E000D1587B68FA6822329200D150FB680133B1
:1053F000FB60FB68072BF0DDBD4604B080BC01BC40
:105400000047C04678A2000880B588B000AFF860B9
:10541000B9607A60FB685B684022D31AFB61FA6965
:105420007B68934200D9131CBB61FB685B6808333F
:10543000FA68D118BA68BB69081C111C1A1C00F064
:1054400051FAFB685A687B68D3183F2B06D8FB6873
:105450005A687B68D218FB685A6035E0FB680833ED
:10546000FA68101C191C0122FFF7C6FC7A68BB6998
:10547000D31A7B607B689B097B61BA68BB69D218D1
:10548000F9687B69081C111C1A1CFFF7B5FCFB6846
:105490001A687B6901339B01D218FB681A607A682D
:1054A0003F231A40FB685A60FB68191C08317B696E
:1054B0009A01BB69D318BA68D218FB685B68081CEC
:1054C000111C1A1C00F00EFABD4608B080BC01BCCD
:1054D0000047C04680B586B000AF786039607B6811
:1054E0001A687B685B68D2187B681A607B681B68E7
:1054F000DB00FB607B685B6809225242D21A3F23C3
:105500001340BB607B685B6879680822C9188A18F9
:10551000802111705A1C7B685A607B685B68083375
:105520007A68D218BB680433101C00211A1C00F0E2
:1055300093FA7B685A68BB68D3181A1D7B685A6057
:105540007B685B68FA68120E1206110E78680822F2
:10555000C018821811705A1C7B685A607B685B689F
:10556000FA68120C1206110E78680822C018821808
:1055700011705A1C7B685A607B685B68FA68120A73
:105580001206110E78680822C018821811705A1C71
:105590007B685A607B685B68FA681206110E78684F
:1055A0000822C018821811705A1C7B685A607B68E8
:1055B0001A1C08327B685B689B097968081C111CFF
:1055C0001A1CFFF719FC00237B6124E003233B61D5
:1055D0001BE07B699A003B69D3183A68D3187A6854
:1055E0007969223189008A581206120E1A703B69B5
:1055F000013B3B617B687A6922329200D358190AD9
:105600007B687A6922329200D1503B69002BE0DA44
:105610007B6901337B617B69072BD7DDBD4606B013
:1056200080BC01BC0047C04680B5AEB000AFF8609A
:10563000B9607A603B1C1033181CFFF7C1FE391C9F
:105640001031FA68BB68081C111C1A1CFFF7DCFE3D
:105650003A1C10327B68101C191CFFF73BFFBD463B
:105660002EB080BC01BC00474A1E08BF7047C0F086
:105670002481884240F21681114200F01781B0FA6D
:1056800080F3B1FA81F2A2EB0303C3F11F0304A27A
:1056900002EB03134FF000029F4600BFAFF3008000
:1056A000B0EBC17F00BF42EB020228BFA0EBC1708C
:1056B000B0EB817F00BF42EB020228BFA0EB8170FC
:1056C000B0EB417F00BF42EB020228BFA0EB41706C
:1056D000B0EB017F00BF42EB020228BFA0EB0170DC
:1056E000B0EBC16F00BF42EB020228BFA0EBC1606C
:1056F000B0EB816F00BF42EB020228BFA0EB8160DC
:10570000B0EB416F00BF42EB020228BFA0EB41604B
:10571000B0EB016F00BF42EB020228BFA0EB0160BB
:10572000B0EBC15F00BF42EB020228BFA0EBC1504B
:10573000B0EB815F00BF42EB020228BFA0EB8150BB
:10574000B0EB415F00BF42EB020228BFA0EB41502B
:10575000B0EB015F00BF42EB020228BFA0EB01509B
:10576000B0EBC14F00BF42EB020228BFA0EBC1402B
:10577000B0EB814F00BF42EB020228BFA0EB81409B
:10578000B0EB414F00BF42EB020228BFA0EB41400B
:10579000B0EB014F00BF42EB020228BFA0EB01407B
:1057A000B0EBC13F00BF42EB020228BFA0EBC1300B
:1057B000B0EB813F00BF42EB020228BFA0EB81307B
:1057C000B0EB413F00BF42EB020228BFA0EB4130EB
:1057D000B0EB013F00BF42EB020228BFA0EB01305B
:1057E000B0EBC12F00BF42EB020228BFA0EBC120EB
:1057F000B0EB812F00BF42EB020228BFA0EB81205B
:10580000B0EB412F00BF42EB020228BFA0EB4120CA
:10581000B0EB012F00BF42EB020228BFA0EB01203A
:10582000B0EBC11F00BF42EB020228BFA0EBC110CA
:10583000B0EB811F00BF42EB020228BFA0EB81103A
:10584000B0EB411F00BF42EB020228BFA0EB4110AA
:10585000B0EB011F00BF42EB020228BFA0EB01101A
:10586000B0EBC10F00BF42EB020228BFA0EBC100AA
:10587000B0EB810F00BF42EB020228BFA0EB81001A
:10588000B0EB410F00BF42EB020228BFA0EB41008A
:10589000B0EB010F00BF42EB020228BFA0EB0100FA
:1058A000104670470CBF012000207047B1FA81F20A
:1058B000C2F11F0220FA02F0704708B14FF0FF302A
:1058C00000F00EB80029F8D02DE90340FFF7CCFE18
:1058D000BDE8064002FB00F3A1EB0301704700BFE7
:1058E000704700BF032A2DE9F00F09D82AB1002321
:1058F000CC5CC45401339342FAD1BDE8F00F704739
:10590000830702440ED0441C4D1C15F8017C04F0A2
:105910000306234601342946013504F8027C002E93
:10592000F3D100E0034611F003046DD0D71A0D1B2C
:10593000032F2E6819DDC4F1040C4FEAC4081C1DA6
:105940004FEACC0C55F8047FC4EB0209234604311E
:105950000434B9F1030F26FA08FA07FA0CFB3E46A5
:105960004BEA0A0744F8087CECDC9A42C5D90133BB
:105970000131013211F8014C01330131934203F836
:10598000024CF7D1B9E70C684033403143F8404C42
:1059900051F83C4C43F83C4C51F8384C43F8384CE7
:1059A00051F8344C43F8344C51F8304C43F8304CF7
:1059B00051F82C4C43F82C4C51F8284C43F8284C07
:1059C00051F8244C43F8244C51F8204C43F8204C17
:1059D00051F81C4C43F81C4C51F8184C43F8184C27
:1059E00051F8144C43F8144C51F8104C43F8104C37
:1059F00051F80C4C43F80C4C51F8084C43F8084C47
:105A000051F8044C43F8044CD41A3F2CBBDC11E091
:105A10000C681033103143F8104C51F80C4C43F81B
:105A20000C4C51F8084C43F8084C51F8044C43F81E
:105A3000044CD41A0F2CEBDC032C96DD1C1D0D1D21
:105A400055F8047C161B2346294604340435032EDE
:105A500044F8087CF4DC88E7032AC9B270B408D89B
:105A60002AB10346121803F8011B9342FBD170BC04
:105A700070478307024409D0441C04F00305234601
:105A800004F8011C0134002DF7D100E00346D51ABB
:105A900001EB01243F2D04EB04442CDD1C6040335A
:105AA000D51A43F83C4C3F2D43F8384C43F8344C5E
:105AB00043F8304C43F82C4C43F8284C43F8244C22
:105AC00043F8204C43F81C4C43F8184C43F8144C52
:105AD00043F8104C43F80C4C43F8084C43F8044C82
:105AE000DCDC08E01C601033D51A43F80C4C43F89A
:105AF000084C43F8044C0F2DF4DC032D08DD1D1D6C
:105B0000561B45F8044C032E2B4605F10405F7DC23
:105B10009A42ACD90133013203F8011C013393429C
:105B2000FAD1A4E7002100F004B80C4B5B584350B5
:105B300004310B480B4B42189A42FFF4F6AF0A4A65
:105B400000F003B8002342F8043B084B9A42FFF4EC
:105B5000F9AF03F019FE00F00DF8704700C100081E
:105B600000000020B8020020B80200209821002088
:105B7000FFF7FEBF2DE9F04F9F4B85B098479F4B35
:105B800098479F4B98479F4B98479F4B98479F4BF1
:105B900098479F4B98479F499F4BF52098479F4EAA
:105BA00042F21070B0479B4820219D4B9847002837
:105BB00040F0AE819B4C9C489649A0479B48954934
:105BC000A0479B489349A0479A489249A0479A4BBF
:105BD000984701228F4840F22551984B9847984B9F
:105BE000984749F2413380B2984240F07181954B19
:105BF0001880954B9847954B9847954B9847954BF0
:105C000000259847944C954B9847DFF8A882284682
:105C100029464FF4A072F0230095C0470194904CA0
:105C2000904F2A46182032214FF6E0730095DFF896
:105C30008892B847DFF884B22A46782034214FF69C
:105C4000E07300950194B8472A4618204B214FF67F
:105C5000E0738DE82002B847DFF864A218206421C1
:105C6000744A4FF6FF738DE82008D047182078213A
:105C70007D4A4FF6FF738DE82008D0477B4C1820F3
:105C8000B4217B4A4FF6FF738DE82008D047794B4B
:105C900098472388642523F0080323807649013D33
:105CA0008847ADB24FF6DC70B047002DF6D123889F
:105CB00003F0080292B25AB16C4A23F00803138031
:105CC0006D4A9047238803F008039BB2002BF7D05E
:105CD0004FF6FF750020694E01464FF4A072F02385
:105CE0000095C0470196664E1420472100221F23CD
:105CF0000095B8478C20462100224FF478438DE868
:105D00006000B8475F4E002213468DE8200218203D
:105D10007321B84701965C4E1420B42100224FF441
:105D200078430095B8475A20B22100224FF47843B7
:105D30008DE86000B8470095544D00225A20C821D4
:105D40004FF478430195B847514D524B524E984706
:105D500000234FF47A72514F2A803370DFF864A128
:105D6000DFF86491DFF864819B461BE003F00403D5
:105D70009BB223BB3378002B26D12388D9072BD4A1
:105D8000E388002B31D1C8472A88034612B9C207DD
:105D900000F1AA8003F008039BB2002B40F09F8023
:105DA0003F48C047D0473B88D807DFD53D4B984791
:105DB0003A490B8803F004039BB2002BDAD03A4A2D
:105DC00090473378002BD8D0334B384983F800B054
:105DD00088472388D907D3D5244A23F001031380A9
:105DE000254B9847E388002BCDD0314988471F4A7F
:105DF000A2F806B0C7E700BF515F0008D95F0008EE
:105E0000AD9F00088993000841600008796100088F
:105E1000D96100080038014085600008D170000891
:105E2000459D0008A960000898A30008D8A30008B1
:105E3000C4A30008B0A30008D1950008A99B0008DE
:105E4000C5690008C202002085740008616100086D
:105E5000C9600008116100081C020020416D0008A3
:105E60001002002049750008ECA00008040300207F
:105E7000A4A300085D760008C97700082802002066
:105E800034020020E0010020F8010020EC01002095
:105E9000C6020020257F0008C4020020E402002082
:105EA00020030020ED8D0008F9890008651C00081A
:105EB0008982000859740008400200200402002072
:105EC000A574000885350008A93300081D96000850
:105ED000144B9847144B49F225321A8089E6134A2D
:105EE0009047134B98475BE710490390884704207D
:105EF000104A90471049884780B21228039B03D963
:105F00000E4928220A8045E70D4A9047039B41E746
:105F10000C480D4B9847F5287FF44CAE0B4B984737
:105F200048E600BFD96A0008C20200207186000856
:105F30002D2E0008DD340008A1300008C602002024
:105F4000651C000800380140FD9C0008D98300084A
:105F50001C4B1D4910B519601C49002259601521C0
:105F60009A60DA601A6159610721D96144F63D618E
:105F700099611A625A621A6812F4003F5A681DD079
:105F800022F003025A605A6842F001025A605A68CD
:105F900042F480325A600B4C0D4B4CF2503023606F
:105FA0000C4B984723689B0107D5636823F00303D4
:105FB0006360636843F00203636010BD22F48032C3
:105FC0005A60E8E7001002408100010000841D00D3
:105FD00081000101D1700008104B30B45A6810489C
:105FE00022F0E0625A605D680E4945F000755D6020
:105FF0000D4B4FF6FF7203600C4B0D4C43604FF09E
:106000003333C2600B600B4B4B600B4BCA60636059
:106010000A4BE26044221A6030BC70470000014025
:1060200000080140000C0140303343B3B44834331E
:10603000001001403B4384880000303300140140CD
:1060400010B5002384B00C4CADF80430ADF8063028
:10605000ADF80830ADF80C300C23694620464FF4FB
:106060001642ADF80A30054B0092984720460121B0
:10607000034B984704B010BD0038014075990008E3
:10608000399B000870B5064D06460C462046802117
:10609000A8470028FAD020463146024B984770BDE9
:1060A000459D0008A19C000870B5044600780D4687
:1060B00030B1044E2946B04714F8010F0028F9D139
:1060C00070BD00BF85600008104B80201880002242
:1060D0004FF440509A801A819A811A829A821883CA
:1060E00010209A83188440F60F609A840521188541
:1060F00009209885998619879A87A3F84020A3F8E4
:106100004820A3F84C2081221A80704700040040E8
:10611000124B80211980002246F260019A801A8178
:106120001A829A821A8399834FF48851198440F60F
:10613000FF719A841A859985A1F500619A861A875C
:106140009987A1F58061A3F84010A3F84820A3F82F
:106150004C209A8181221A80704700BF00080040BD
:10616000034B00229A6007221A60024A5A60704765
:1061700010E000E040190100104B002240F6FF71D2
:106180001A605A609A60DA601A615A619A61DA613B
:106190001A6259629A62DA621A635A639A639A6857
:1061A000194642F004029A608B68044A5807FBD5EE
:1061B000936843F001039360704700BF00280140DB
:1061C0004163836843F00103836003689B07FCD548
:1061D000C06C80B2704700BFF8B59C4E4FF400779A
:1061E00041F288309A4D3761A8474FF6E850776101
:1061F000A8470A2437614FF6FF70A847631E13F0C3
:10620000FF04F8D1934B4FF4005290484FF480466E
:106210005A615E61C4684FF4004104F47F4444F065
:10622000CF04C460596119611E611A615A611E610F
:10623000C768642407F47F47C760596119611A6110
:106240005A611E61C76807F47F4747F0C107C760FE
:10625000596119611A615A611E61C76807F47F4765
:1062600047F03007C760596119611A615A615E6170
:10627000C76807F47F4747F0ED07C76059611961A8
:106280001E611A615A611E61C76807F47F4747F0B3
:106290006707C760596119611A615A611E61C76851
:1062A00007F47F4747F00307C760596119611A6116
:1062B0005A611E61C76807F47F4747F01207C7603D
:1062C000596119611A615A611E61C76807F47F47F5
:1062D00047F08107C760596119611A615A615E61AF
:1062E000C76807F47F4747F0CB07C760596119615A
:1062F0001E611A615A611E61C76807F47F4747F043
:106300003907C760596119611A615A611E61C7680E
:1063100007F47F4747F02C07C760596119611A617C
:106320005A611E61C76807F47F47C76059611961E8
:106330001A615A611E61C76807F47F4747F0340746
:10634000C760596119611A615A611E61C76807F413
:106350007F4747F00207C760596119611A615A61A6
:106360005E61C76807F47F4747F0EA07C760596175
:1063700019611E611A615A611E61C76807F47F477F
:10638000C760596119611A615A611E61C76807F4D3
:106390007F47C760596119611A615A615E61C768B8
:1063A00007F47F4747F0E807C760596119611E612C
:1063B0001A615A611E61C76807F47F4747F0850775
:1063C000C760596119611A615A611E61C76807F493
:1063D0007F4747F00A07C760596119611A615A611E
:1063E0001E61C76807F47F4747F07807C7605961A7
:1063F00019611A615A615E61C76807F47F4747F007
:10640000F707C760596119611E611A615A611E61FF
:10641000C76807F47F4747F02007C76059611961D3
:106420001A615A615E61C76807F47F4747F0C00789
:10643000C760596119611E611A615A611E61C7689E
:1064400007F47F4747F02607C76005E0000C0140CE
:10645000D170000800100140596119611A615A6138
:106460005E61C76807F47F4747F0C107C76059619D
:1064700019611E611A615A611E61C76807F47F477E
:1064800047F00107C760596119611A615A615E617D
:10649000C76807F47F4747F0C507C76059611961AE
:1064A0001E611A615A611E61C76807F47F4747F091
:1064B0002B07C760596119611A615A611E61C7686B
:1064C00007F47F4747F02F07C760596119611A61C8
:1064D0005A615E61C76807F47F4747F0C707C76026
:1064E000596119611E611A615A611E61C76807F41A
:1064F0007F4747F0C707C760596119611A615A6140
:106500005E61C76807F47F4747F03A07C760596183
:1065100019611E611A615A611E61C76807F47F47DD
:1065200047F05507C760596119611A615A615E6188
:10653000C76807F47F4747F03607C760596119619C
:106540001E611A615A611E61C76807F47F4747F0F0
:106550002007C760596119611A615A615E61C76895
:1065600007F47F4747F0B107C760596119611E61A1
:106570001A615A611E61C76807F47F47C760596195
:1065800019611A615A611E61C76807F47F4747F0B5
:106590001807C760596119611A615A615E61C7685D
:1065A00007F47F4747F0B607C760596119611E615C
:1065B0001A615A611E61C76807F47F4747F00A07EE
:1065C000C760596119611A615A611E61C76807F491
:1065D0007F4747F0E207C760596119611A615A6144
:1065E0005E61C76807F47F4747F0F207C7605961EB
:1065F00019611E611A615A611E61C76807F47F47FD
:10660000C760596119611A615A615E61C76807F410
:106610007F4747F02607C760596119611E611A61FB
:106620005A611E61C76807F47F4747F00107C760DA
:10663000596119611A615A615E61C76807F47F4741
:1066400047F0E007C760596119611E611A615A611C
:106650001E61C76807F47F4747F00F07C76059619D
:1066600019611A615A611E61C76807F47F4747F0D4
:106670001D07C760596119611A615A611E61C768B7
:1066800007F47F4747F01A07C760596119611A611B
:106690005A611E61C76807F47F4747F00907C76062
:1066A000596119611A615A611E61C76807F47F4711
:1066B00047F00F07C760596119611A615A611E617D
:1066C000C76807F47F4747F00907C7605961196138
:1066D0001A615A611E61C76807F47F4747F0460791
:1066E000C760596119611A615A611E61C76807F470
:1066F0007F4747F08807C760596119611A615A617D
:106700001E61C76807F47F4747F03907C7605961C2
:1067100019611A615A611E61C76807F47F4747F023
:106720000507C760596119611A615A611E61C7681E
:1067300007F47F4747F00F07C760596119611A6175
:106740005A611E61C76807F47F4747F00307C760B7
:10675000596119611A615A611E61C76807F47F4760
:1067600047F00707C760596119611A615A611E61D4
:10677000C76807F47F4747F00507C760596119618B
:106780001A615A611E61C76807F47F47C760596183
:1067900019611A615A615E61C76807F47F4747F063
:1067A000E107C760596119611E611A615A611E6172
:1067B000C76807F47F47C760596119611A615A6158
:1067C0001E61C76807F47F4747F02207C760596119
:1067D00019611A615A611E61C76807F47F4747F063
:1067E0002507C760596119611A615A611E61C7683E
:1067F00007F47F4747F00607C760596119611A61BE
:106800005A611E61C76807F47F4747F01007C760E9
:10681000596119611A615A611E61C76807F47F479F
:1068200047F00607C760596119611A615A611E6114
:10683000C76807F47F4747F03907C7605961196196
:106840001A615A611E61C76807F47F4747F0220743
:10685000C760596119611A615A611E61C76807F4FE
:106860007F4747F04A07C760596119611A615A6149
:106870001E61C76807F47F4747F00A07C760596180
:1068800019611A615A611E61C76807F47F4747F0B2
:106890001007C760596119611A615A611E61C768A2
:1068A00007F47F4747F00C07C760596119611A6107
:1068B0005A611E61C76807F47F4747F03807C76011
:1068C000596119611A615A611E61C76807F47F47EF
:1068D00047F03A07C760596119611A615A611E6130
:1068E000C76807F47F4747F00F07C7605961196110
:1068F0001A615A615E61C76807F47F4747F0110764
:10690000C760596119611E611A614CF25030A84785
:10691000631E13F0FF040E4EF7D10E4B4FF40052DE
:106920004FF480410C4D5A615961EF684FF40044B7
:1069300007F47F4747F02907EF604CF250305C6165
:106940001C6119611A61B0474CF25030B047F8BD74
:10695000D170000800100140000C01400A4B70B4D7
:106960004FF400524FF48041084D5A615961EE686E
:106970004FF4004406F47F463043E8605C611C61DC
:1069800019611A6170BC704700100140000C014091
:106990000A4B30B44FF40052094C4FF480415A6115
:1069A0001961E5684FF4004105F47F452843E06034
:1069B000596119611A6130BC704700BF0010014075
:1069C000000C0140204B2DE9F0474FF400514FF4EB
:1069D0008042DFF87C9059615A61D9F80C504FF42D
:1069E000004405F47F4545F0D305C9F80C505C61BF
:1069F0001C611A61196159611A614FF044336420B6
:106A0000DFF85080C9F80030C04740270F4E0425FA
:106A10000024BA460A20C6F814A0C047D9F80820B6
:106A20006B1ED2B213F0FF05376142EA0424F1D1A4
:106A3000074B4FF033321A604FF400522046C3F830
:106A40001024BDE8F08700BF00100140000801409D
:106A5000000C0140D17000082DE9F84F1B4C1C4D73
:106A60004FF400574FF480498246DFF868800220D7
:106A70006761C4F814908B46C047EB684FF400463A
:106A800003F47F4343EA1A23EB6066612661EB68F7
:106A9000022003F47F434AEA0303EB606661266148
:106AA000C4F81090C047EB6803F47F4343EA1B230C
:106AB000EB6066612661EB6803F47F434BEA0303F6
:106AC000EB60666126612761BDE8F88F0010014028
:106AD000000C0140D1700008F8B57E4C4FF40075F1
:106AE00041F288307C4F2561B84765614FF6E85028
:106AF000B8470A24013C4FF6FF70A4B2B847002CF7
:106B0000F8D1744B4FF400721A610A25013D4FF61B
:106B1000FF70ADB2B847704E002DF7D141F288300A
:106B20006E4CB047E52047F6F001A04701204FF436
:106B30008071A04702204FF4E061A0470320382174
:106B4000A04704202946A047082040F20721A0477B
:106B500009202946A0470A202946A0470C2029469B
:106B6000A0470D202946A0470F202946A047102006
:106B70002946A04711200721A04712202946A047F7
:106B800029461320A04707200121A04720210720E4
:106B9000A0474CF25030B0474CF25030B0474CF266
:106BA0005030B047102041F29021A04740F22121FF
:106BB0001120A0474CF25030B0474CF25030B04753
:106BC0004CF25030B04781211220A0474CF2503097
:106BD000B0474CF25030B0474CF25030B047132021
:106BE0004FF4A851A04729200C21A0470D212B20AC
:106BF000A0474CF25030B0474CF25030B0474CF206
:106C00005030B04720202946A04721204FF4807102
:106C1000A047302040F20331A04731200621A04791
:106C200032200121A04735204FF40171A0473620C2
:106C30000421A047372040F20741A04738202946C9
:106C4000A047392040F20441A0473C2040F20241D5
:106C5000A0473D200421A04750202946A047EF210E
:106C60005120A04752202946A047532040F23F110F
:106C7000A04760204FF41C51A04761200121A0478C
:106C80006A202946A04780202946A047812029461E
:106C9000A04782202946A04783202946A047842078
:106CA0002946A04785202946A04790201021A047CB
:106CB00092204FF4C061A04740F233110720A04753
:106CC0004CF25030B0474CF25030B0474CF250309C
:106CD000B047F8BD000C0140D1700008596A0008A7
:106CE000F8B50F4C4FF400530E4E63614FF48043E0
:106CF00002200D4F6361B847F3684FF4004503F479
:106D00007F43F360022065612561B847F36803F4AF
:106D10007F4343F02203F36065612561F8BD00BF46
:106D200000100140000C0140D1700008024B4FF4EC
:106D300000521A61704700BF00100140704700BF49
:106D400070B5002182B04FF00060194B98470024C5
:106D50000126184D1B2301A88DF804308DF805403D
:106D60008DF806408DF80760A847122301A88DF81A
:106D700004308DF805408DF806408DF80760A8476F
:106D80000B2301A88DF804308DF805408DF80640DE
:106D90008DF80760A847252301A88DF804308DF8E9
:106DA00005408DF806408DF80760A84702B070BD19
:106DB0002D9900088598000810B5064B9847064B9A
:106DC0000446984704F50063044A03EB800090876B
:106DD00010BD00BFC1320008C134000800080040E7
:106DE00008B5074B9847074A074B1018D96810F8A1
:106DF000022C21F01E0102F01E020A43DA6008BDD7
:106E0000192F0008E8A3000800080140F8B5124C4B
:106E10004FF4806663684FF4006723F47043636047
:106E200063680E4D43F4405363600A202761666136
:106E3000A8470A202661A8470A206761A8470A20B8
:106E40006661A847636823F470436360636843F432
:106E500080436360F8BD00BF000C0140D1700008A2
:106E6000F8B5124C4FF4806663684FF4006723F462
:106E70007043636063680E4D43F4405363600A20BF
:106E800067616661A8470A202661A8470A20276132
:106E9000A8470A206661A847636823F470436360CB
:106EA000636843F480436360F8BD00BF000C014099
:106EB000D17000082DE9F0471C4D1D4C6B6807464A
:106EC00023F470436B606B68082643F440536B6097
:106ED0004FF40069A2464FF480683A064CBFC5F8EB
:106EE0001090C5F814900A20A0470A20C5F8108019
:106EF000A0470A20A0470A20012EC5F814800B4B9A
:106F000008D0013E7F00D04716F0FF06FFB2E4D163
:106F1000BDE8F0875A6822F470425A605A6842F419
:106F200080425A60024B9847BDE8F087000C014050
:106F3000D17000082DE9F0410F4C104E4FF00808B9
:106F40004FF480670A20A0470A203761A047B36842
:106F50006D000A20EDB2190548BF45F00105A047B4
:106F60000A207761A04708F1FF3313F0FF08E9D149
:106F70002846BDE8F08100BFD1700008000C014038
:106F8000F8B50A4D0A4C0A204FF48066A0470A2043
:106F90002E61A047AF680A20A0470A206E61A04773
:106FA00087F40060C0F3C020F8BD00BF000C0140B2
:106FB000D170000870B5114C114D63680A2023F49C
:106FC0007043636063684FF4806643F440536360CA
:106FD0004FF400636361A8470A202661A8470A208E
:106FE000A8470A206661A847636823F4704363607A
:106FF000636843F48043636070BD00BF000C0140D0
:10700000D170000870B5114C114D63680A2023F44B
:107010007043636063684FF4806643F44053636079
:107020004FF400632361A8470A202661A8470A207D
:10703000A8470A206661A847636823F47043636029
:10704000636843F48043636070BD00BF000C01407F
:10705000D17000082DE9F0410D4EDFF840804FF46B
:1070600080650C4CC047092735610A20A0470A20DB
:107070003561A0470A20A0470A207561A0477B1E02
:1070800013F0FF07F1D1C047034B9847BDE8F081EB
:10709000000C0140D1700008616E00080D6E000800
:1070A000044B5A6822F470425A605A6842F4804293
:1070B0005A607047000C0140044B5A6822F4704239
:1070C0005A605A6842F440525A607047000C0140BE
:1070D00082B0ADF80600BDF806309BB24BB1BDF8EA
:1070E0000630013BADF80630BDF806309BB2002BF0
:1070F000F5D102B0704700BF0132520002F0FE022B
:10710000531EDBB230B40024012B8C540DD900F097
:107110000F04E2B2092A94BF44F0300237325D1EF8
:10712000CA54EBB20009012BF1D15A1E7820C85481
:10713000D2B2302308468B5430BC70472DE9F84357
:107140000646104F2A201546884699460E4CB847E9
:10715000300AA047F0B2013E4644B6B2A047300A1A
:10716000A047F0B2A0472B20B847280AA047E8B2B2
:10717000013D4D44ADB2A047280AA047E8B2A04760
:10718000BDE8F8835D690008916900082DE9F843BE
:1071900087B2204C0E465220394691469846BDF89B
:1071A0002050A047791E4944B6B2532089B2A04767
:1071B00050203146A047711E4144512089B2A0475A
:1071C00020203146A04721203946A047124B98473E
:1071D00009FB08F311484FF480420261B3B1104C2F
:1071E0002E0A4FF40041EDB2E268013B02F47F4207
:1071F00046EA0202E26041610161E26802F47F4214
:1072000045EA0202E26041610161EDD1054B984718
:10721000BDE8F883596A0008E16C000800100140DD
:10722000000C01402D6D00082DE9F047099C8146B6
:10723000A088E57A0730521BC01000FB02FE94F8CC
:1072400006A022682C4D0E46522049460AFB0E2A03
:107250001F46BDF82080A847A18853200139494422
:1072600089B2A84750203146A847A1795120013959
:10727000711889B2A84721204946A84731462020E5
:10728000A8471E4B98471E494FF480430B61A279D3
:10729000A38802FB03F3C3F3CF0343B3013B1FFAFD
:1072A00083FC18480AF1FF3ED4444FF400421EF814
:1072B000014F0825C36814F0800F0CBF46463E46B8
:1072C00003F47F4343EA1623C3604A610A61C3683B
:1072D000F6B203F47F43013D64001E4315F0FF0541
:1072E000C660E4B24A610A61E4D1E645DFD1064BEB
:1072F0009847BDE8F08700BF596A0008E16C0008B4
:1073000000100140000C01402D6D0008F8B5174633
:107310001E468AB280B2B9B29BB2194CBDF8185061
:10732000A04718484FF48042174C4FF40053436174
:107330004261E16807FB06F301F47F4646F02C0644
:107340004FF40041E6604161016102619BB12E0A88
:10735000EDB2E268013B02F47F4246EA0202E260DB
:1073600041610161E26802F47F4245EA0202E260A3
:1073700041610161EDD1034B4FF400521A61F8BD38
:107380003D71000800100140000C01402DE9F84358
:10739000099C8C46A188E67ACD1D921BED1005FB59
:1073A00002FEA6792568624606FB0E551F46334647
:1073B000264EBDF82080B04725494FF4804325482C
:1073C0004FF400524A614B61C6684FF4004206F424
:1073D0007F4646F02C06C6604A610A610B61A388AD
:1073E000A47904FB03F3C3F3CF0343B3013B1FFAB8
:1073F00083FCAC446B1E13F8014F0825D0F80C90A9
:1074000014F0800F0CBF46463E4609F47F4949EA16
:107410001629C0F80C904A610A61D0F80C90F6B2B7
:1074200009F47F49013D640046EA090615F0FF05AD
:10743000C660E4B24A610A61E0D16345DBD1044B26
:107440004FF400521A61BDE8F88300BF3D71000897
:1074500000100140000C014070B5074C82B0258837
:10746000BDF8186049F24134A54200960CBF034CA8
:10747000034CA04702B070BDC20200200D7300088B
:107480008D71000810B5002382B01846009319468C
:107490004FF4A072F023024CA04702B010BD00BF11
:1074A000597400082DE9F04F244C85B09846BDF87A
:1074B00038302688039349F241339E420446894678
:1074C00017460F9D1DD0DFF878B040F23F1A17F82D
:1074D000016B20464946434632467EB1039E0195E4
:1074E0000096D8472B89E418A4B25445EFD9AB7A5B
:1074F000002409EB030C1FFA8CF9E8E705B0BDE89E
:10750000F08FDFF840A017F801BB204649464346FC
:107510005A46BBF1000FF1D0039E01950096D0476B
:107520002B89E418A4B240F23F139C42EBD9AB7A0A
:10753000002409EB030C1FFA8CF9E4E7C2020020D7
:10754000297200088D73000870B5084C82B0258838
:1075500049F24134A542BDF81860079C0096019499
:107560000CBF034C034CA04702B070BDC202002008
:107570008D73000829720008F8B52B4E2B4B0020A4
:107580002B4D984700213089A8472A4B0720984760
:107590000721B088A847284B002098470021F08891
:1075A000A847264B1220984712213088A847244B21
:1075B000002098470021B089A847224B0020984717
:1075C0000021F089A847204B002098470021308AED
:1075D000A8471E4B4FF4806098471D4C4FF48061C4
:1075E000B08AA847A047400896381A4B00B298477F
:1075F0007788A0474008A0F1960189B23846A8478D
:10760000154B0020984700217089A847F08A002177
:10761000A84706F11A04323634F8020F0021A847B1
:10762000B442F9D1F8BD00BF6C020020B12F0008B0
:10763000E9940008A12E0008352F00083930000811
:1076400039310008B531000855320008DD32000834
:1076500031330008BD3000086934000830B583B00C
:107660000C200DF106013F4CA047BDF806304FF24B
:10767000A535AB421DD03C4B98473C4B2946188B57
:107680003B4B98473B4B98473B4B98473B4B984766
:107690003B4A012111803B4A0621D1813A4A00230D
:1076A00013803A4A13803A4A13803A4A138003B04F
:1076B00030BD2E4D0DF106012889A047364BBDF98E
:1076C000060098470DF10601A888A047334B9DF9A5
:1076D000060098470DF10601E888A047304B9DF958
:1076E000060098470DF106012888A0472D4B9DF90B
:1076F000060098470DF10601A889A0472A4B9DF97D
:10770000060098470DF10601E889A047274B9DF92F
:10771000060098470DF10601288AA047244BBDF9C1
:10772000060098470DF10601A88AA047214BBDF835
:10773000060098470DF106016888A047BDF90600CC
:107740001D4B98471D4B98470C300DF1060135F83D
:107750001000A047BDF90600194B9847E88A19495F
:10776000A0478FE725930008797500086C02002078
:10777000E9940008B96D0008E16D0008DD17000804
:10778000C0020020040300209A2100209C21002038
:107790009821002000030020B12F0008A12E00082E
:1077A000352F00083930000839310008B53100089C
:1077B00055320008DD320008BD300008192F0008DE
:1077C00069340008E4020020F8B5654D654C4FF6B9
:1077D000FF774FF088330A2067802B60624B984711
:1077E000AE68AB6846F47F4646F00706B6B24FF087
:1077F0003332BE422A6003F0030E5BD023886680DA
:1078000043F008032380A188564B8E4257D0258829
:1078100045F0020323804FF6EF7399423ED0534B5D
:1078200001E08A423BD01A8818460433002AF8D176
:10783000002225F006055A23A680A28122826382B7
:107840002580A38A4A494EEA830303F00F028A5C2B
:10785000A382012A434B28D0FF2A1AD0052145488C
:10786000454B9847B0F5106F11D8B0F5407F34BF45
:1078700002240024414D2B78A34207D02046404BE0
:10788000984702203F4B2C709847F8BDF8BD012463
:10789000F0E70E22DA8001221A81DFE73A48837886
:1078A000C278E38063812281C2E70F22DA8000225E
:1078B0001A81D3E76688BE42A5D1A188A7E79A8935
:1078C000D989013292B28A429A8123D9C81C824254
:1078D000B7D1188A5D8A421C92B2954299811A8268
:1078E000AFD11A884FF6FD7702F0040117408AB233
:1078F0001F80AAB14FF6EF739E4229D01B4B01E0C7
:10790000964226D01A8819460433002AF8D104304A
:10791000608296E795D11A8842F002021A8090E7B9
:107920004FF6FE713140114B01E091420AD01A88A6
:107930001D460433002AF8D147F00407153027808C
:1079400060827EE7AB78EA78E38063812281F3E7A7
:107950000D498B78CA78E38063812281D7E700BF25
:10796000000C014004030020D1700008B4BF0008DF
:1079700084BE000800280140C1610008E702002021
:10798000352F0008DD340008B0BF000808B50A4BE9
:10799000984780F0040000F00403DBB23BB9074BCA
:1079A0009847074B98470220064B984708BD064B5F
:1079B0009847064B9847F6E7A933000819340008A2
:1079C000651C0008DD340008C13300087D2E000866
:1079D00030B54F4B83B09847062820D8DFE800F039
:1079E00004395385627724004A4B984701304A4B4B
:1079F00040B29847494C0546494B9847A9B2494B74
:107A0000A0880C3598470DF10601474B34F8150056
:107A10009847464BBDF906009847454B9847454C5B
:107A20000220A04703B030BD434B984701300346C6
:107A3000ADF8063000B2414B9847384A034681B250
:107A40001089ADF80630374B98473A4C0420A047D0
:107A5000E6E73B4B984701303A4B40B298472F4BF3
:107A6000044681B218882F4B98470D2CCCBF364B5B
:107A7000364B0A3CE4B29847032C43D8344B0F22D0
:107A8000DA812C4CCCE7334B98470130324B40B273
:107A90009847224B81B29889224B98472A4B9847A6
:107AA000244CBDE72D4B984702300346ADF8063015
:107AB00000B22B4B9847194A034681B2ADF8063005
:107AC000108A184B98471A4B98471A4CA8E7254B31
:107AD000984701380346ADF8063000B2224B98476C
:107AE0000E4A034681B25088ABE7204B98470130DD
:107AF0001F4B40B29847094B81B2D889094B984730
:107B00000C4C8DE7124B0622DA810A4C88E700BF45
:107B100091330008192F0008A12E00086C020020E4
:107B2000E16D0008E9940008259300086934000815
:107B3000B96D0008DD3400081D300008B12F0008C1
:107B4000A130000839300008651C0008FD1B000842
:107B5000040300209931000839310008C1320008BF
:107B6000553200081D310008BD30000839320008C8
:107B7000B531000830B5484B83B09847062820D867
:107B8000DFE800F004394B6F5A7C2400434B9847E0
:107B90000138434B40B29847424C0546424B984708
:107BA000A9B2424BA0880C3598470DF10601404B15
:107BB00034F8150098473F4BBDF9060098473E4BF7
:107BC00098473E4C0220A04703B030BD3C4B98473D
:107BD00001380346ADF8063000B23A4B9847314AB7
:107BE000034681B21089ADF80630304B9847334CCC
:107BF0000420A047E6E7344B98470138334B40B2A6
:107C00009847284B044681B21888284B98470C2C7B
:107C10000EDC2F4B9847294CD4E72E4B9847013860
:107C20002D4B40B298471F4B81B298891F4B984704
:107C30002A4B9847214CC5E7294B98470238034601
:107C4000ADF8063000B2274B9847164A034681B27A
:107C5000ADF80630108A154B9847174B9847174CCC
:107C6000B0E7214B98470138204B40B298470D4B65
:107C700081B2D8890D4B9847104CA3E71C4B98470D
:107C800001300346ADF8063000B21A4B9847054A5A
:107C9000034681B25088A6E791330008192F0008E7
:107CA000A12E00086C020020E16D0008E994000894
:107CB0002593000869340008B96D0008DD34000818
:107CC0001D300008B12F0008A1300008393000082D
:107CD000FD1B00089931000839310008651C0008B7
:107CE000C13200085532000839320008B5310008A9
:107CF0001D310008BD30000830B50F4C0F4A2388F5
:107D000083B083F0010323801946D08A0C4B984737
:107D1000238813F001040CD1CD20142164225023B8
:107D20000094084DA84700940F2014218C2246236C
:107D3000A84703B030BD00BFE40200206C02002061
:107D4000E99400085974000808B5064B9847064B9B
:107D500000280CBF0620002098470220034B9847BC
:107D600008BD00BF9133000849330008DD34000826
:107D700008B5064B9847064B01280CBF052001208B
:107D800098470220034B984708BD00BF9133000875
:107D900049330008DD34000808B5074B984702381E
:107DA000C0B202289ABF054B185C0220044B9847CA
:107DB0000220044B984708BD91330008C4BE000858
:107DC00049330008DD3400082DE9F04F2A4B87B015
:107DD00098472A4B02909847294B01909847294B86
:107DE00003901220984702250020274B274EDFF8EA
:107DF000BC80274FDFF8B8B0DFF8B8A0254C984713
:107E00004FF000092846C047B8474EF66020D847D3
:107E1000D047ADF81690A047C307ADF81600FAD5C5
:107E20001D4B9847A0F5007083B201351946ADF897
:107E3000163036F8020F194BEDB2984768B20E288B
:107E4000E1D1104B029898470198C0470E4B039818
:107E50009847B847019B0DF1160103F10C02104B36
:107E600033F812000F4B9847BDF916000E4B984798
:107E700007B0BDE8F08F00BFA1300008192F00083F
:107E80009931000839300008393100088602002095
:107E9000E16D0008A93300084D340008E99400089A
:107EA0006C0200202593000869340008A12E000808
:107EB000D1700008651C000808B5074B9847A0F56D
:107EC000967000EBD070054B40F34F0098470220AE
:107ED000034B984708BD00BF31330008BD30000890
:107EE000DD34000808B50A4BB3F90020094BB3F99B
:107EF0000030D31803EBD37358108000064B00B248
:107F00009847064B98470220054B984708BD00BF8D
:107F1000C8020020DE02002055320008B96D0008BA
:107F2000DD34000838B5154B4FF40042144C5A614B
:107F30003225013D4FF6E850ADB2A047002DF8D1F3
:107F40000E4B4FF400421A613225013D4FF6E850C6
:107F5000ADB2A047002DF8D1084B4FF400425A6152
:107F60003225013D4FF6E850ADB2A047002DF8D1C3
:107F7000024B4FF400421A6138BD00BF00080140B7
:107F8000D17000082DE9F04FDFF8BC8185B00024E6
:107F90000E202146544A40F23F538DE81001534FC2
:107FA000B847534B9847DFF8A4915248C847042874
:107FB00005461BD08DE810010E2021464E4A1F2396
:107FC000B8474E4CFA204E49A04700204C49A047E4
:107FD000E8B24B49A047F0204949A047C6F3072023
:107FE0004749A047F0B24649A047FEE74548C84781
:107FF00004280546DED14448C8470428054607D072
:108000008DE810010E202146404A1F23B847D8E7CB
:108010003F4BDFF83CB11D68D8470246C0B1DFF8DE
:108020003491DFF834A1AB1E2646C5EB090909EBF4
:10803000030033F8021F03920293D047711C0428F7
:108040000546039A029B3ED18EB29642EFD101E0E3
:10805000DFF804A1D8472F4C2F4B208098472F4B97
:10806000608098472E4BA08098472E4BE080984721
:108070002D4B208198472D4B608198472C4BA08138
:1080800098472C4BE08198472B4B20829847DFF88C
:1080900078906082002604EB090303F17843A3F58E
:1080A000684348461988D047731C0428054609F1DF
:1080B000020910D19EB20A2EEDD102201F4B984723
:1080C00005B0BDE8F08F00218DE802010E201C4AAA
:1080D0001F23B84775E700218DE802010E20194AD9
:1080E0001F23B8476DE700BFC8BE0008A57400088D
:1080F000AD9F000800E00008D0BE000885600008C1
:108100000038014000E4000800E80008D8BE00087C
:1081100090210020E8020020192F0008952F000868
:10812000A13000089931000839320008C132000836
:108130001D3100081D300008C1340008DD3400087E
:10814000E0BE0008E8BE0008040200207DA0000890
:108150003133000802E0000811A0000810B5002427
:1081600082B0214600942B4C2B4A40F23F530E2004
:1081700001942A4CA0472A4B18882A4B98472A4B2F
:1081800093F90000294B9847294B93F90000294B9C
:108190009847294B93F90000284B9847284B93F9AF
:1081A0000000284B9847284B93F90000274B98472D
:1081B000274BB3F90000274B9847274BB3F9000032
:1081C000264B9847264BB3F90000264B9847264B81
:1081D000B3F90000254B9847254B1C68254B984761
:1081E00068B1411E89B201F1806101F5E041224B85
:1081F000490033F8022F8B4224F8022BF9D11F4B90
:1082000098471F4B98471F4C0220A0470420A047C7
:1082100002B010BD04020020F0BE0008A5740008E2
:1082200000E80008DD32000802E80008A12E00087E
:1082300004E80008352F000806E800083930000877
:1082400008E80008393100080AE80008B5310008DC
:108250000CE80008553200080EE80008BD300008A0
:1082600010E80008B12F000812E80008693400087F
:108270009021002031330008FEDF0008C1330008E0
:108280007D2E0008DD34000810B5334B82B0DB884A
:10829000013B102B1AD8DFE803F036393C3F42454A
:1082A000484B194E51191B54572009002B4B1A8863
:1082B00082F0040202F0040189B21A8031B90091FF
:1082C0000F20C52170221023254CA04702B010BDFD
:1082D000244B9847244B01221A70204B1A8802F035
:1082E000040189B20029F1D082F0020202F00201F9
:1082F00089B21A8000292AD01C4B1D4A5A604FF4BB
:1083000080525A61E2E71B4B9847DFE71A4B9847C8
:10831000DCE71A4B9847D9E7194B9847D6E7194B32
:108320009847D3E7184B9847D0E7184B9847CDE7C5
:10833000174B9847CAE7174B9847C7E7164B98471C
:10834000C4E7164B9847C1E7154B9847BEE7154A57
:10835000064B5A60BAE700BF04030020E402002085
:108360005974000879750008C4020020000C01400F
:108370003B438388497D0008717D0008997D000892
:108380008D790008C97D0008B97E0008E57E0008E7
:10839000F97C00085D810008857F0008D17900081C
:1083A000757B00083B43848838B5094B4FF4004285
:1083B00004465A6138B1074D013C4FF6E850A4B26B
:1083C000A847002CF8D1024B4FF400421A6138BD87
:1083D00000080140D17000082DE9F04F894B8A4D0B
:1083E0008A4C2B608A4B4FF6FF476B604FF6FF734A
:1083F000EB604FF044332360864B83B0864E63605E
:108400004FF6DC70E760B04747F65573EB604FF608
:10841000DC70E760B0474FF6DC70B0474FF6DC70B9
:10842000B0474FF6DC70B047A36847F6EB6203F045
:10843000FB07522F14BF4FF4007700271FFA83FB6E
:10844000D904714B714CDA604FF6FF5348BF47F0C7
:108450003007E3604FF6DC7048BFBFB2B0474FF65D
:10846000DC70B047A3686D4C03F0FB02A92A18BF6B
:1084700047F400771FFA83FADA04694B58BF47F0D4
:1084800030079847674B9847674B984749F2413305
:1084900080B2984278D12080644D654B4FF000083F
:1084A0009847DFF8C491634902222088C847624C8C
:1084B00018207821614A4FF6FF73CDF800800195AE
:1084C000A0475F4A4FF6FF7398207821CDF80080CF
:1084D0000195A0475B4B41465B48984755490222AE
:1084E000C84718208C21594A4FF6FF73CDF80080F9
:1084F0000195A0474FF6FF738C21514A9820CDF883
:1085000000800195A0474B4902223846C847CDF864
:10851000008001951820B4214D4A4FF6FF73A04703
:10852000002F37D14FF4FC6300979820B421444AC0
:108530000195A047474B0526A3F801603146C227A5
:10854000502618461F701E71434A444B98471E2000
:10855000434B98473749022200265846C8474FF4F4
:10856000FC632821364A982000960195A04731499E
:1085700002225046C8470096019598203C21304A77
:108580004FF4FC63A047FEE7364B984749F225338A
:10859000238081E71F239820B421294ACDF8008049
:1085A0000195A0472B4B052739464FF0C20EA3F883
:1085B00001704627184683F800E01F71264A274BB2
:1085C0009847274F0A20B8474FF00F0808F1FF38A7
:1085D0004FF6DC701FFA88F8B047B8F1000FF5D1FC
:1085E0000A20B8474FF00F0808F1FF384FF6DC704B
:1085F0001FFA88F8B047B8F1000FF5D10A20B84744
:10860000A8E700BF3033333300080140000C0140BD
:10861000B344343333438488D1700008C20200204D
:10862000D95F0008D9610008C5690008040200206C
:1086300085740008E8020020A5740008F8BE000850
:10864000EA020020C16100080028014008BF0008BC
:1086500014BF000898030020003801400997000863
:10866000A9830008D96A0008F9700008000000001A
:108670002DE9F04F9C4E89B0B0479C4B81469847FE
:108680000746002800F0A081DFF8AC820022D8F86D
:1086900000A04FEA400C40F6FF751446104696467F
:1086A0003AF8023024B2C9EB03031BB22DB20232F6
:1086B0009C42B8BF1C469D42A8BF1D46A3F5007151
:1086C00062459E4401FB0100EAD1894A21B202922F
:1086D000138840F6FC729142A4B203DC2AB2032A4A
:1086E00000F35F81ADB223F00401A4F50073A5F59A
:1086F0000072641B029D29807E4D9EFBF7F92B8042
:108700007D4BA9F500711A807C4BDFF830A21980EF
:108710007B4B7C491C8088477A4A04463846904700
:1087200001462046D047DFF818B2D847764B984725
:10873000764B9847764B1FFA89F41880B047D8F8E3
:10874000002004F108051188083C091AB1F5007FE2
:10875000B4BF00210121002F00F02B81002300264F
:1087600024B201938446023A01370123B04628B26D
:10877000059409E00136012E00F00381CDF80C903C
:1087800001210133BB4210D032F8025F0CB2CCEBB6
:108790000505012C03F1FF392DB200F0DB80A84262
:1087A000E8DD01330021BB42EED1012E40F3FD8014
:1087B000029D09B22B88012943F002032B8000F0AF
:1087C000FE80049A069B079D9A42C2EB050408F1BD
:1087D000FF3000F3E1804B4988474A4A064620466D
:1087E0009047074639463046D0474A4C8046A04716
:1087F000DFF85091013859F82010474D4046A847FE
:10880000DFF8448103460146C8F800304FF07E503F
:10881000D047424B3B491860019888473146009049
:10882000D0470646A047013859F820103046D047B7
:10883000009B3B4A394610601846D0473949A84743
:10884000394A3A4BD8F8009010600022384F484619
:1088500038491A80B847012408B90EE03446354932
:108860004846D047631C334981469EB2B84700282A
:10887000F4D12E4AC8F8009014802849DFF8CCA023
:108880000C680423AAF800302046D84714A3D3E983
:108890000023DFF8BC90C847E8B1214905270E68DE
:1088A00000E0474623492046A8472249044630466F
:1088B000A8477B1C064620461FFA83F8D84708A322
:1088C000D3E90023C8470028EBD1144BAAF8007065
:1088D0001C60134C266009B0BDE8F08FAFF3008038
:1088E0007B14AE47E17A843FC1340008313300087D
:1088F00000030020C8020020DE020020D002002079
:10890000FE0200201910000879020008B50D0008C9
:10891000DA020020A1300008C11000081C0300206A
:10892000CC0200200000C842E0020020DC0200204F
:108930002514000800007A44902100202912000824
:10894000D9070008ECBF0008D4020020D80200209C
:10895000790D0008059CAC42FFF613AF049D08F1A9
:108960000108B8F1010F08BF4D46049586B1039C7C
:10897000019DC4EB09016D180195CDF81C900021F3
:10898000FFE6CDF818904C46CDF80C903146F8E64D
:10899000CDF81C903146F4E6019D9B1AED18019527
:1089A00019E7ADB243F004019FE6B8F1010F3FF7BC
:1089B000FFAE029A138823F0020313808BE7039A19
:1089C000069B701ED41A06E7084B4FF2010402936F
:1089D0001B88029D43F004032B8040F6FF524FF4A6
:1089E0007E43BE46DFF8088086E600BF0003002015
:1089F00090210020AFF30080114B10B51B8882B08E
:108A000003F002039BB26BB94FF4784300930D4B14
:108A10000F200193C5210C4A4FF6FF730B4CA04762
:108A200002B010BD4FF478430093064B0F20019322
:108A3000C521074A4FF6FF73044CA047F0E700BF7B
:108A4000E40200200402002030BF0008A5740008E2
:108A500020BF0008234AF0B4A2FB0032520BC2EB45
:108A6000C203C3EB4313C2EB031300EB03101E4B13
:108A700080B2A3FB00439B09C3EB831403EB841474
:108A800003EB440400EBC400184E84B2A6FB0406BA
:108A90007609F0B2C0EB402500EB8505C0EBC500C0
:108AA00004EB8000124D80B2A5FB0045ED08ECB24E
:108AB000C4EB4437C4EB870400EB440043F03003BD
:108AC00042F0300246F0300645F0300540F030000C
:108AD0004B70002308710A708E70CD704B71084680
:108AE000F0BC70475917B7D1D34D62101F85EB51B9
:108AF000CDCCCCCC000000002DE9F843404B04461F
:108B00000E4698473F4B804620469847DFF8109125
:108B10003D4FC84736A3D3E90023B8473B4BA8F1E4
:108B20000202044653F822000D46C84702460B468F
:108B300020462946B84730A3D3E90023B847344B31
:108B400098470021334B0446984700283BD02046E5
:108B5000314B9847202480B2711C304B9847B8F1B4
:108B6000090F10DCF2783179737832712E22F270AD
:108B70005622B2710022302B7171F2712AD03470FA
:108B80003046BDE8F8837179B278307931716D2162
:108B9000F578717156212023B1710021302A33708C
:108BA0007270B570F070F1711AD1EAB2302A737038
:108BB0001AD1C2B2302AB37018D1F3700323F4541F
:108BC0003046BDE8F88304F10040134B98472D244C
:108BD00080B2C1E72023747033703046BDE8F8835B
:108BE0000123013B5BB2EAE70223FAE70323F8E73C
:108BF0000000000000C8E93FE9263108AC1CF03F46
:108C0000192F0008191000088108000894BE0008F8
:108C1000050E0008251400084D140008558A0008A8
:108C2000D9070008AFF30080F0B44E1E0924D4B178
:108C30002246012303EB8303013A5B0012F0FF029B
:108C4000F8D1013CB0FBF3F2E4B242F03007FF2C64
:108C5000D2B206F8017F03FB1200E8D100238B7229
:108C60000846F0BC704740F030057570F6E700BF6D
:108C70002DE9F04F8B4689B01E460021544B8046AB
:108C800017469847002840F096804FF00009DFF81B
:108C900054A14046D04702AC0DF109014D4B019063
:108CA00098472146002211F8010F531C3028154621
:108CB0005FFA82FC1A4604D10A2BF4D11D46944671
:108CC0000B2302A8C218BBF1000F7CD008A8C31860
:108CD00013F8181C30290BD1202003F8180C531C52
:108CE00001E003F8010C1A4613F8011B3029F8D0F3
:108CF0002E295CD0BCF10A0F54D0B9F1000F4AD034
:108D000008A901EB050B2D230BF8183CB7B98DF81A
:108D100013701BF8183C337063B1314600230133E4
:108D2000DBB208A8C218521912F8182C01F8012F4A
:108D3000002AF4D1304609B0BDE8F08F2E238DF81B
:108D400013300198244B9847244B014640469847DE
:108D5000DFF894800246B94610462149C04709F120
:108D6000FF3919F0FF090246F6D1D04705A9194B82
:108D700098477B1E0DF10902DBB2C7F11601D2182C
:108D8000635C01349442E372FAD108A9CF1900233D
:108D900007F80C3CBDE708AB03EB050B20230BF8F1
:108DA000183CB3E730238DF812300925A5E73023AE
:108DB00002F8013C9EE741460020084B98474FF0DF
:108DC0000109804663E708A9CB1813F8181C8FE740
:108DD000FD130008298C000811100008AD0E0008D2
:108DE000000020414D140008C11000082DE9F04F8B
:108DF000704D85B000264FF29E79DFF80C826E4CE4
:108E00006E4ACD2014214B46009601956C4FB8F860
:108E100000A0A0476B4BDFF8F4B13946B3F900006E
:108E2000D8470AF0040A1FFA8AFAB24514BFCA46A4
:108E30004FF01F0A02461421F72053460096019571
:108E4000A047614ACD2024214B4600960195A047BA
:108E50005E4B3946B3F90000D847242102465346F9
:108E6000F72000960195A047594ACD2034214B4662
:108E700000960195A047574B3946B3F90000D847F3
:108E8000342102465346F72000960195A047524AE6
:108E9000CD2044214B4600960195A0474F4B3946C3
:108EA000B3F90000D847442102465346F720009604
:108EB0000195A0474A4ACD2054214B460096019582
:108EC000A047484B3946B3F90000D8475421024621
:108ED0005346F72000960195A0470F201421424ADF
:108EE0004B4600960195A0470F2024213F4A4B4650
:108EF00000960195A0470F2034213D4A4B4600962D
:108F00000195A0473B4A4B46009601950F2044210E
:108F1000A047B8F8003003F0020292B2002A77D1DD
:108F200003F008039BB2002B00F0038100263920D8
:108F30001421314A4FF29E7300960195A0473920C3
:108F400024212D4A4FF29E7300960195A0473920A7
:108F50003421294A4FF29E7300960195A04700964E
:108F6000019539204421244A4FF29E73A047234B98
:108F70001B8803F0040292B26AB103F002039BB2B1
:108F800063B94FF478438DE828000F20C5211C4AAF
:108F90004FF6FF73A04705B0BDE8F08F4FF478435C
:108FA0008DE828000F20C521164A4FF6FF73A04711
:108FB000F1E700BF04020020A574000840BF0008CC
:108FC000E8020020C802002048BF0008DE0200209E
:108FD00050BF0008D002002058BF0008FE02002049
:108FE00060BF0008DA02002068BF000870BF0008F8
:108FF00078BF00087CBF000888BF0008E40200209A
:1090000030BF000820BF000800030020F98A0008D4
:10901000624803210A463B460068DFF8ACA1D0470E
:109020005F4B604A1B88384652F823105E4B9847C6
:10903000DFF898913846C847DFF894B11FFA80FCF2
:10904000BBF800309C45C0F08280002639201421F6
:10905000564A4FF29E7300960195ABF800C0A047A8
:10906000534803210A46514B0068D047514A4F48A4
:1090700013884C4ADFF85CB152F823104A4B9847EA
:109080004A48C847BBF800301FFA80FC9C4578D39B
:10909000002639202421454A4FF29E7300960195FF
:1090A000ABF800C0A047444803210A463F4B006884
:1090B000D047404A3D4813883A4ADFF81CB152F87D
:1090C0002310394B98473948C847BBF800301FFA7E
:1090D00080FC9C4548D3002639203421334A4FF286
:1090E0009E7300960195ABF800C0A047334803215A
:1090F00001222E4B0068D0472C48C847304B86468B
:10910000B3F800A093F8029007EB000C00960195CD
:109110004FF29E7327F80EA039204421234A8CF881
:109120000290A047B8F8003023F00803A8F80030F8
:109130001DE700933920462314217822214EB047A1
:10914000B8F8003043F00803A8F80030EEE6DA0083
:109150000096CDF80CC03920142112B21023194EFC
:10916000B047DDF80CC070E7DA000096CDF80CC00F
:109170003920342112B21023124EB047DDF80CC052
:10918000A9E7DA000096CDF80CC03920242112B2EC
:1091900010230C4EB047DDF80CC079E7D402002054
:1091A000DC0200204C02002011010008E80200202F
:1091B0001C030020D8020020CC020020E002002086
:1091C00084BF000859740008718C00081902000857
:1091D0009A2100209C21002098210020704700BF88
:1091E000FEE700BFFEE700BFFEE700BFFEE700BFEF
:1091F000704700BF704700BF704700BF0C4B1A8814
:10920000013A92B25AB11A800A4B1A8832B1013A25
:1092100092B21A8012B9084B01221A707047074A9D
:1092200002201188188041F001031380ECE700BF91
:10923000C0020020C6020020C40200200403002057
:1092400000B5094883B040F22551084B984740B11A
:10925000074B0548984702A901F8010D054B064840
:10926000984703B000BD00BF00380140ED9D0008E5
:10927000FD9C0008A5950008200300201A4B70B53E
:109280001A8803F580631B8805469BB292B2E3B946
:109290004EF6EE63D21A18BF01229402531C134AF1
:1092A0009B0204F1006404F570449A18944203D3BD
:1092B0000EE00434A2420BD923680133F9D12046D1
:1092C0000B4EB04704280BD070BD1AB1AB2070BD57
:1092D000802070BD4EF6EE629B1A5A425A41DCE77E
:1092E000A01C2946B04770BD00F00008FEEF000842
:1092F00011A0000810B50748074CA047042800D06B
:1093000010BD00210348054B98470428F8D10448B4
:10931000A047F5E700F000087DA0000811A00008B4
:1093200000F40008124B134A1B8812889BB210B439
:1093300092B2A3B112B1AB2010BC70470E4B0F4CD0
:109340001A46128892B2824204D10CE01A8892B274
:10935000824208D0043BA342F8D80120ECE7084B36
:10936000084C1A46EDE733F8023C00200B80E3E797
:1093700000F0000800F40008FEF7000802F40008FE
:10938000FEF3000802F000082DE9F0474B4E4C4F69
:1093900033884EF6EE623C889BB29342A4B249D029
:1093A0004FF6FF75AB4236D01BB1464B9847BDE830
:1093B000F087002CF9D0AC4268D0434E434FDFF821
:1093C00010A1DFF81C81DFF81C911C463A8836F8A2
:1093D000023B92B29A4208BF254618462BB29C42E5
:1093E0003B4904F1010409D0C047012806D036F8F2
:1093F000020CBAF80010C84704285BD11B2CE5D139
:1094000000212F48334B98470428D0D1324B2B48AA
:109410009847BDE8F087002CF8D09442C5D130467B
:109420002D4B98470428C2D138460021294B984734
:10943000BDE8F087002C2ED1234E284FDFF890A0F6
:10944000DFF89C80DFF89C904FF6FF753A8836F87D
:10945000023B92B29A4208BF254618462BB29C4264
:109460001B4904F1010409D0C047012806D036F891
:10947000020CBAF80010C84704281DD11B2CE5D1F6
:1094800000210E48134B9847042890D1124B0C48EA
:109490009847BDE8F0874FF6FF739C4285D1384668
:1094A0000D4B9847042882D130460021094B98473C
:1094B000BDE8F087BDE8F087BDE8F08700F0000860
:1094C00000F40008F59200086C02002006F4000881
:1094D0009E21002011A000087DA0000806F00008D1
:1094E000259300087D9200082DE9F84F244C05468D
:1094F0000E46A047802801D0BDE8F88F214A224BB4
:109500001188188889B280B219B1002832D0AB20F6
:10951000F2E790461F4638464EF6EE61DFF874904B
:10952000C8470428E8D128463146A0470428E3D19B
:10953000DFF864B0DFF864A00BF136063BF8022BCD
:1095400012499542104609D0D047012806D00F4B4A
:109550003BF8020C1988A04704280ED1B345EDD181
:1095600040460B4B98470428C6D138460021C847CF
:10957000BDE8F88F98461746CDE7BDE8F88F00BFE5
:109580007D92000800F0000800F400089E210020F1
:109590007DA0000811A000086C020020259300089F
:1095A000704700BF10B443690A781A70026A4369B1
:1095B000848E013314190169A34228BF13469942CE
:1095C00003D04361012010BC70470020FBE700BFBF
:1095D0000C4B322230B40C499A86DA861A870B4A31
:1095E0000B4859629961D961DA630A490A4A002431
:1095F000254618621861586199621C861A649C732A
:1096000030BC7047200300206403002069970008E5
:10961000FC03002030040020A1950008D0F814C0FD
:10962000F8B50446FF260125FE2723699C4532D064
:10963000216AA08E13F8012B0818834228BF0B461D
:10964000FE2A236134D0A37B03F04001C9B219B3D1
:1096500003F0200123F04000C9B2A07300292CD0F0
:10966000002A2AD1228EA16A531C9BB28F542386D2
:10967000A26AB2F801209A4202D9228F9A423AD2C3
:10968000E36B9847A37BD4F814C023F02003A373A3
:1096900023699C45CCD1F8BD03F02003DBB2002B3D
:1096A000C3D0218EA06A4B1C9BB242542386DFE7B5
:1096B000A37B43F04003A373B7E7E42A12D00BD88F
:1096C000102A05D3122A0DD9A2F1E001022909D9E5
:1096D00023F06003A373A8E7F22A0FD8EF2A01D280
:1096E000E92AF5D1A36A1A70A36A9E70A37B258626
:1096F00043F02003A373D4F814C096E7FC2AF1D0FA
:1097000023F06003A37390E72DE9F8430E468046EB
:109710001446D1B1124D20468021A8470028FAD026
:109720002046FE21DFF83C90C84720468021A8470C
:109730000028FAD018F8017B20463946C847FE2F8A
:1097400005D0013EB6B2002EEFD1BDE8F883204629
:109750008021A8470028FAD020460021C847F0E71A
:10976000459D0008A19C000808B504480378EF2B2C
:1097700003D14178024A034B984708BD30040020CA
:1097800000380140099700083B4B3C4A186800210B
:1097900040F001001860586882B002405A601868B2
:1097A0001A4620F0847020F480301860186820F485
:1097B00080201860586820F4FE0058604FF41F00A5
:1097C000986000910191196841F48031196003E0BB
:1097D000009BB3F5A06F09D0136803F40033019325
:1097E000009B01330093019B002BF1D0224B1B689F
:1097F00013F4003306D001230193019B012B05D004
:1098000002B070470193019B012BF9D11C4A1A4BFE
:109810001068194640F010001060106820F0030036
:109820001060106840F0020010605A685A605A6870
:109830005A605A6842F480625A605A6822F47C1274
:109840005A605A6842F4E8125A601A6842F080720C
:109850001A600B68084A9B01FBD55368114623F038
:1098600003035360536843F0020353604B6803F0F3
:109870000C03082BFAD1C3E7001002400000FFF8E8
:109880000020024038B5C3780446012B03D9234891
:109890007421234B984763780F2B39D8A3780F2B6B
:1098A00031D8E3785BB92378012103F01F0201FA74
:1098B00002F15B091B4A203342F8231038BD1A4BD2
:1098C0006078DB680F22DB43C3F30223C3F104019A
:1098D00022FA03F300FA01F0A578217803EA0502E1
:1098E000024301F16043120103F5614383F8002351
:1098F0002378012103F01F0201FA02F1094A5B09F2
:1099000042F8231038BD7621054B04489847C8E734
:109910007521034B01489847C0E700BF4CC00008C1
:109920003D6D000800E100E000ED00E0B0F1005FF7
:1099300038B504460D4606D0B0F1006F03D0094893
:109940009D21094B9847094B9D4203D905489E210B
:10995000054B984725F0604525F07F05044B2C43C7
:109960009C6038BD4CC000083D6D0008FEFF0F0034
:1099700000ED00E070B5684B86B0984204460D4695
:1099800013D0A3F5744398420FD003F58063984237
:109990000BD003F58063984207D003F580639842AB
:1099A00003D05E48B5215E4B98472B685D4A013B6A
:1099B000934200F29A80AB8833B1B3F5805F03D055
:1099C0005648B721564B9847EB8863B1B3F5805F93
:1099D00009D0B3F5005F06D0B3F5405F03D04F4820
:1099E000B8214F4B98472B894BB1B3F5806F06D008
:1099F000B3F5C06F03D04948B921494B98476A89EC
:109A00004FF6F373134003BBFAB1AB8923B3B3F53D
:109A1000807F0BD0B3F5007F08D0B3F5407F05D031
:109A20003F4B3E48BB219847AB89ABB13A4A944281
:109A300012D03D4A94420FD03C4A94420CD0BF21F0
:109A40003648374B9847A98907E0354B3348BA2148
:109A50009847AB89002BDAD11946228AEB8822F489
:109A600040521204120C1A432282A3892E89AA881A
:109A700023F4B053688923F00C031B0432430243E0
:109A80001B0C1343A381A38A01A823F440731B0476
:109A90001B0C0B43A382264B98471F4B9C42A38968
:109AA00008BF04991BB218BF0399002B22DB28685A
:109AB00001EB810101EB81018000B1FBF0F21D4956
:109AC000A089A1FB025300B25B091E016425002896
:109AD00003FB152317DB1B013233A1FB0351C1F339
:109AE00043113143218106B070BDB6210C4B0B48A8
:109AF000984760E72B6801EB810101EB81015B0076
:109B0000B1FBF3F2DBE7DB003233A1FB0321C1F34E
:109B100042113143E6E700BF003801407CC0000835
:109B20003D6D00081FAA440000440040004800406A
:109B3000199F00081F85EB5138B5184B0446984211
:109B40000D4614D0A3F57443984210D003F58063FA
:109B500098420CD003F58063984208D003F58063E7
:109B6000984204D00E4840F25F110E4B9847012DE9
:109B70000AD94FF4B0710A480A4B9847A3899BB29F
:109B800043F40053A38138BD002DF7D1A38923F4FA
:109B900000531B041B0CA38138BD00BF00380140DB
:109BA0007CC000083D6D00083A4B70B598420546F0
:109BB0000C46164614D0A3F57443984210D003F512
:109BC000806398420CD003F58063984208D003F577
:109BD0008063984204D030484FF4C3712F4B9847AC
:109BE000282C1ED040F227739C421AD040F22663E4
:109BF0009C4216D040F225539C4212D040F224439E
:109C00009C420ED040F646039C420AD003F5927364
:109C10009C4206D0602C04D01F4840F287111F4B95
:109C20009847012E04D91C484FF4C4711B4B984728
:109C300040F66A139C421AD004F01F030122C4F3B9
:109C40004214944202FA03F30FD0022C06D01435CA
:109C50002A683EB922EA03032B6070BD10352A68DA
:109C6000002EF7D013432B6070BD0C35F0E7094B85
:109C70009D420CD0A3F574439D4208D003F5806348
:109C80009D4204D04FF4C6710348044B98474FF4EB
:109C90008063DCE7003801407CC000083D6D0008AF
:109CA00038B5134B044698420D4614D0A3F57443BF
:109CB000984210D003F5806398420CD003F580637E
:109CC000984208D003F58063984204D0094840F2D6
:109CD0004F21094B9847B5F5007F04D305484FF451
:109CE0001471054B9847E905C90DA18038BD00BF27
:109CF000003801407CC000083D6D00080E4B10B5D7
:109D00009842044614D0A3F57443984210D003F54A
:109D1000806398420CD003F58063984208D003F525
:109D20008063984204D005484FF41871044B98475B
:109D3000A088C005C00D10BD003801407CC00008DF
:109D40003D6D000838B5254B044698420D4614D0A9
:109D5000A3F57443984210D003F5806398420CD069
:109D600003F58063984208D003F58063984204D0DD
:109D70001B4840F26A311B4B9847012D18D0802DAB
:109D800016D0402D14D0202D12D0102D10D0B5F5A6
:109D9000807F0DD0B5F5007F10D0082D08D0042DA0
:109DA00006D0022D04D040F26B310D480D4B984780
:109DB00023881D420CBF0020012038BD074B9C4268
:109DC000F6D0094B9C42F3D003F580639C42EFD060
:109DD00040F26F31034B02489847E9E700380140F1
:109DE0007CC000083D6D00080044004038B5464B7B
:109DF000044698420D4614D0A3F57443984210D0FF
:109E000003F5806398420CD003F58063984208D034
:109E100003F58063984204D03C4840F2BD313C4B8E
:109E20009847282D4CD040F227739D423BD040F2FA
:109E300026639D4237D040F225539D4233D040F2F5
:109E400024439D422FD040F646039D4244D003F563
:109E500092739D4245D0B5F5587F34D0B5F5187F43
:109E600031D0B5F5B07F2ED040F2BE31284B274817
:109E700098470121C5F3421205F01F038A4201FAF7
:109E800003F315D0022A28D0A08A80B21840238874
:109E90009BB2A0B101222D0A02FA05F51D420CBFAA
:109EA0000020012038BD05F01F03012202FA03F350
:109EB000A08980B2184023889BB20028EAD138BD1F
:109EC0004FF48073F4E705F01F03012202FA03F355
:109ED000A08A80B21840DAE74023208A80B2184076
:109EE000D5E7094B9C420BD00A4B9C4208D003F5A6
:109EF00080639C4204D040F2C2310448044B98472E
:109F00004FF48063E4E700BF003801407CC00008E4
:109F10003D6D0008004400401F4910B44B6803F039
:109F20000C03042B01D0082B22D01C4A02601A4BD0
:109F30001B495C68C4F303140C5D22FA04F242600E
:109F40005C68C4F302240C5D22FA04F484605C684B
:109F5000C4F3C224095D22FA01F2C2605B681149B0
:109F6000C3F38133CB5CB2FBF3F2026110BC7047E8
:109F70004A684B68C2F383420232DC0307D54B6860
:109F80009B0304D4054B03FB02F20260CFE7064BB0
:109F900003FB02F20260CAE70010024000127A00DE
:109FA000A8020020A402002000093D00034B044A3F
:109FB0005A6002F188325A60704700BF00200240A8
:109FC00023016745084BDA68D2070BD4DA685007DB
:109FD00001D502207047DB6813F0100F0CBF04207E
:109FE00003207047012070470020024038B5074D1C
:109FF0000446A847012804D12CB1A847013C0128F8
:10A00000FAD004B138BD052038BD00BFC59F000897
:10A01000154AF8B500F17843934204460E4606D837
:10A020004FF40050114DA84704280BD0F8BD40F262
:10A030008B310F4B0F4898470C4D4FF40050A847F9
:10A040000428F3D10C4F4FF400503B6943F0010357
:10A050003B612680A8470528E8D03A6941F6FE739F
:10A0600013403B61F8BD00BFFEFF0F00ED9F0008ED
:10A070003D6D0008B8C0000800200240164B00F1FA
:10A0800078429A4270B5044606D84FF43020134DFA
:10A09000A84704280BD070BD4FF4D371104B114862
:10A0A00098470E4D4FF43020A8470428F3D10E4EA8
:10A0B0004FF43020336943F0020333617461336934
:10A0C00043F040033361A8470528E4D0326941F6E4
:10A0D000FD731340336170BDFEFF0F00ED9F00085C
:10A0E0003D6D0008B8C00008002002404C49423ACB
:10A0F0002031353030332D30343500000A00DD009A
:10A10000280012006E00DD0032001200BF00DD00EA
:10A11000280012000001DD0010001200323056004D
:10A120000031305600003556000000325600000065
:10A130003156000000302E355600302E3256003099
:10A140002E31560035306D560032306D56003130AC
:10A150006D5600356D56000000007A440000FA4349
:10A1600000007A430000C842000048420000C84195
:10A17000000020410000A040000020400000803F7F
:10A180000000003F0000803E4443000041430000C7
:10A19000474E4400353030730000323030730000D9
:10A1A00031303073000035307300000032307300FE
:10A1B000000031307300000035730000000032737E
:10A1C00000000000317300000000302E35730000E5
:10A1D000302E32730000302E3173000035306D7335
:10A1E000000032306D73000031306D730000356D4A
:10A1F00073000000326D73000000316D73000000C9
:10A20000302E356D7300302E326D7300302E316D6F
:10A2100073003530757300003230757300003130D3
:10A220007573000000000000000000004155544F0D
:10A23000004E4F524D0053494E470000486F6C642A
:10A240006F66660057616974696E6700547269676A
:10A250006765640000F8E007FF0700002020202069
:10A260002020202000000000484F4C440000000047
:10A2700052756E6E696E670067E6096A85AE67BBE8
:10A2800072F36E3C3AF54FA57F520E518C68059BD8
:10A29000ABD9831F19CDE05B982F8A429144377167
:10A2A000CFFBC0B5A5DBB5E95BC25639F111F15959
:10A2B000A4823F92D55E1CAB98AA07D8015B83129B
:10A2C000BE853124C37D0C55745DBE72FEB1DE8047
:10A2D000A706DC9B74F19BC1C1699BE48647BEEF76
:10A2E000C69DC10FCCA10C246F2CE92DAA84744A01
:10A2F000DCA9B05CDA88F97652513E986DC631A877
:10A30000C82703B0C77F59BFF30BE0C64791A7D555
:10A310005163CA0667292914850AB72738211B2EDD
:10A32000FC6D2C4D130D385354730A65BB0A6A76C5
:10A330002EC9C281852C7292A1E8BFA24B661AA8D1
:10A34000708B4BC2A3516CC719E892D1240699D6E1
:10A3500085350EF470A06A1016C1A419086C371E5A
:10A360004C774827B5BCB034B30C1C394AAAD84E38
:10A370004FCA9C5BF36F2E68EE828F746F63A57873
:10A380001478C8840802C78CFAFFBE90EB6C50A406
:10A39000F7A3F9BEF27871C60A0D44534F205368F3
:10A3A000656C6C00426F6F74696E672E2E2E000014
:10A3B00046573A203131332D31353030312D30355B
:10A3C000350000000A0D5757572E4A59455445434A
:10A3D000482E434F4D0A0D000A0D4A594520546539
:10A3E0006368204C74642E00060A000E0C08161ACE
:10A3F000101E1C18020000000000000000000000F9
:10A400000001E0000000000F000FFF8FBFFC0FFFF6
:10A41000800000E0007F00000700038F030E0C0C9B
:10A4200071800000E0001C01C007000387060E04D5
:10A430000C71800000E0001C01C007000387840E3F
:10A44000000870800000E0001C01C0070003838842
:10A450000E1000700F80F8EF001C07F8FF0003815A
:10A46000D00E30007018C39CF3801C01C1C70003DC
:10A4700081F00FF0007038E31CE3801C01C38700FB
:10A480000380E00E3000703FE71CE3801C01C387AF
:10A4900000E380E00E100070380700E3801C01C369
:10A4A0008700E380E00E020070380700E3801C099B
:10A4B000C3870CE380E00E060070382704E3801C9D
:10A4C00019C3871EC700E00E0E00701C4388E3808E
:10A4D0001C39C1C71E3C03F83FFE01FC0F81F1F798
:10A4E000C07FF8F8FF8C00001F8001B0DF8FC00133
:10A4F000801FC001999F8FC0018018C001999803E7
:10A5000000018018DB018F18030E39B01F9B018FEB
:10A510001F831F7DF81F9B01861F831B6D9818CA20
:10A520000D8618031F619818CA0D861803186D98B8
:10A530001FCE0F861F831B7D981F8E07061F830E5D
:10A540003998000400000000000000001C0000001A
:10A5500000000000001800000000000000000000E3
:10A56000000000000000000000018000000000006A
:10A570000000038000003C0F300003C000000FFF0C
:10A58000C0000007C000007C0E780003C000001F60
:10A59000FFF000000FC00001FC0EE00383C1E000EB
:10A5A0003FC3F000001FE00003FFEE0007FFFFE0E5
:10A5B000003C07F800003CFC00007CFFF807FFFFB0
:10A5C000F000007FC00000783F8007FCE7000783B1
:10A5D000C0E000003E000001F61FF80FFFE7700723
:10A5E00083C0E000003C000007EF87FF067C677037
:10A5F00007FFFFE007FFFFFFE07FC7F1FF01FCE778
:10A60000E00383C1E00FFFFFFFE07F03E0FE01FFF7
:10A61000EFE00383C1E00FF81E7FE01800003C016B
:10A62000FCFFC003C3FFE00F001E07C000FFFF00D8
:10A6300003FCF7F003FFFFE000001E000001FFFF36
:10A640000003FECEF803FFFFC000001E000001C0A3
:10A650001F0007BFD87C01C3C00000001E0000001F
:10A66000001E000F07FC300003E001C0001E0000C8
:10A6700000003C003F00FFF80001FC0F80003E009E
:10A6800000000078003E001FFF8000FFFF80387E42
:10A6900000000001F000000007FF80007FFF001FA6
:10A6A000FE00000007E000000000FF00001FFE00A9
:10A6B00007F80000000780000000003C000001F8DF
:10A6C0000000C000000000000000000000000000CA
:10A6D00000000003800000000000000000000001F6
:10A6E0008000000000018000000000000000000069
:10A6F0000001800003000001800000000000000055
:10A7000000000000000003000001800000000000C5
:10A71000799FCCFE6703BCE3C7C3C1E1B800F07802
:10A72000773831898C4C6201984663066331CC01DD
:10A7300098CC39CC31898C4C6201984C630C6631D1
:10A740008C031986318C1AD0D686B4018C8FE30F16
:10A75000E6018C030186318C1AD0D686B4018C8C2C
:10A76000030C06018C030186318C0C606303180115
:10A77000870C030C06018C030186318C0C6063038B
:10A7800018618706230623118C6188CC318C0C60FC
:10A79000630318618203C1C3C1E3DE60F0787BDE2E
:10A7A0000000000000018200000000000000000026
:10A7B000000000000000000D1C0000000000000070
:10A7C0000000000000000000000E18000000000063
:10A7D0000000000000000000003FF8000000000042
:10A7E0000000000000000001E00F000FE00000008A
:10A7F000000003F80FE0030001C00C60000000003F
:10A800000003180C600E0000E00C60000000000067
:10A8100003180C600C0000700C60000000000003C6
:10A82000180C60181FF0380C6000000000000318BE
:10A830000C6018701E180C60000000000003180C5B
:10A840006030C0071C0C60000000000003180C60A2
:10A850003180030C0C60000000000003180C603114
:10A8600080018C0C60000000000003180C60318037
:10A8700001FC0C63FC00007FC003180C6031C000B9
:10A88000000C6E070001C07003180C6030E000007F
:10A890000C78038007001C03180C60383C00000C87
:10A8A0007000C00E000E03180C601807E0000C606A
:10A8B00000C01C000703180C601C003E000CC7F011
:10A8C00060183F8303180C600E0007800C1C386072
:10A8D00030E0E183180C60038000E00C1818603150
:10A8E000803183180C6000F000380C300C6031802F
:10A8F0003183180C60003F001C0C300C60630018A2
:10A90000C3180C600001F00C0C600C60630018C3ED
:10A91000180C6000001C0E0C600C6063FFF8C3187C
:10A920000C60000007060C600C60600000C3180C8F
:10A9300060000001860C600C60600000C3180C60B1
:10A940007F8000C60C600C60600000C3180C607152
:10A950008000C60C600C6063FFFFC3180C6071C000
:10A9600000C60C600C6063000003180C6070C0012E
:10A97000C60C600C6033000003180C603860018C5A
:10A980000C600C6031800003180C6038380F0C0C20
:10A99000600C6030E03FC3180C601C0FF81C0C60AA
:10A9A0000C60183FF183180C601E0000180C600C3E
:10A9B000601C000383180C600F0000700C600C60BA
:10A9C0000E000703180C60038000E00C600C6007A9
:10A9D000000E03180C6001F007800C600C6001C0D1
:10A9E0007803180C60003FFC000FE00FE0007FC010
:10A9F00003F80FE00000000000001FE0000003FE6D
:10AA000000003FFFFF000000FFFC60001FFFC000D0
:10AA10003FFFFFF00001FC1FE0007F07F00007FE92
:10AA200003FC0003F00FE000FC01F80001FE00FF52
:10AA30000007F007E003F800FE0001FE007F800F32
:10AA4000E003E007F8007F0001FE003FC00FE001D7
:10AA5000E007F0007F8001FE001FE01FE001E00F33
:10AA6000F0003F8001FE001FE01FE000E01FE0005B
:10AA70003FC001FE000FF01FF000E01FE0003FC0EC
:10AA800001FE000FF81FF000E03FE0003FE001FE94
:10AA9000000FF81FFC00603FC0001FE001FE000730
:10AAA000F81FFF00003FC0001FE001FE0007FC0F81
:10AAB000FFC0007FC0001FF001FE0007FC0FFFF881
:10AAC000007FC0001FF001FE0007FC07FFFE007FB3
:10AAD000C0001FF001FE0007FC03FFFF807FC000E5
:10AAE0001FF001FE0007FC01FFFFC07FC0001FF048
:10AAF00001FE0007FC007FFFE07FC0001FF001FEA9
:10AB00000007FC001FFFF07FC0001FF001FE0007E0
:10AB1000FC0003FFF07FC0001FF001FE0007FC00F7
:10AB2000007FF87FC0001FF001FE0007F830001F13
:10AB3000F83FC0001FE001FE0007F838000FF83FA3
:10AB4000C0001FE001FE000FF838000FF83FE000E2
:10AB50003FE001FE000FF03C0007F81FE0003FC09F
:10AB600001FE000FE03C0007F81FE0003FC001FEBF
:10AB7000001FE03E0007F00FF0007F8001FE001F85
:10AB8000C03E0007F00FF0007F8001FE003F803FD5
:10AB90000007F007F0007F0001FF007E003F800FFC
:10ABA000E003F800FE0003FF81FC003FC01FC0006F
:10ABB000FC01FC003FFFFFE0003BF03F80007F070F
:10ABC000F0003FFFFF000030FFFE00001FFFC0004D
:10ABD0000000000000001FF0000003FE0000000065
:10ABE000FF807A03E000F4F0001EF038E0C60E3873
:10ABF000018C70000E703871C21C1C038470000E32
:10AC0000703831C2180C038477070E703839E03879
:10AC10000E03C07B8D8E703838F8380E01F0739DAE
:10AC2000CE7038383E380E007C739FCE7038390FA6
:10AC3000380E021E739C0E70383907180C020E7302
:10AC40009C0E703871871C1C030E739C0E7038E1CB
:10AC5000C60E38038C738E4E70FF813C03E0027881
:10AC6000FBC79FF81FFFFFFFFFFFFFF83FFFFFFF3E
:10AC7000FFFF00007FFFFFFFFFC007FFFFFFFFFF99
:10AC8000FC00FFFFFFFFFFFFF01FFFFFFFFFFFFFC5
:10AC9000C07FFFFFFFFFFFFF83FFFFFFFFFFFFFFFF
:10ACA00007FFFFFFFFFFFFFF07FFFFFFFFFFFFFEA5
:10ACB00007FFFFFFFFFFFFFE07FFFFFFFFFFFFFF95
:10ACC00003FFFFFFFFFFFFFF01FFFFFFFFFFFFFF8E
:10ACD00080FFFFFFFFFFFFFFC07FFFFFFFFFFFFFC2
:10ACE000C07FFFFFFFFFFFFFC03FFFFFFFFFFFFF32
:10ACF000C03FFFFFFFFFFFFFC01FFFFFFFFFFFFF82
:10AD0000801FFFFFFFFFFFFF003FFFFFFFFFFFF878
:10AD1000003FFFFFFFFFFFE0007FFFFFFFFFFF009F
:10AD200000FFFFFFFFFFF00001FFFFFFFFFC00003F
:10AD300003FFFFFFFC00000007FFFFFF0000000013
:10AD40000FFFFFFF000000003FFFFFFF00000000BB
:10AD5000FFFFFFFF00000007FFFFFFFF0000003FB5
:10AD6000FFFFFFFE000000FFFFFFFFFC000007FFEA
:10AD7000FFFFFFF8000000000000000000000000DE
:10AD800000000000000000000000000000000000C3
:10AD900000000000000000000000000000000000B3
:10ADA00000000000000000000000000000000000A3
:10ADB0000000000000000000000000000000000093
:10ADC0000000000000000000000000000000000083
:10ADD0000000000000000000000000000000000073
:10ADE0000000000000000000000000000000000063
:10ADF0000000000000000000000000000000000053
:10AE00000000000000000000000000000000000042
:10AE10000000000000000000000000000000000032
:10AE20000000000000000000000000000000000022
:10AE30000000000000000000000000000000000012
:10AE40000000000000000000000000000000000002
:10AE500000000000000000000000000000000000F2
:10AE600000000000000000000000000000000000E2
:10AE700000000000000000000000000000000000D2
:10AE800000000000000000000000000000000000C2
:10AE9000000000000000183C3C3C1818180018186E
:10AEA000000000000066666624000000000000004C
:10AEB000000000000000006C6CFE6C6C6CFE6C6CA2
:10AEC0000000000018187CC6C2C07C060686C67C3E
:10AED0001818000000000000C2C60C183060C686BA
:10AEE000000000000000386C6C3876DCCCCCCC76EE
:10AEF0000000000000303030600000000000000062
:10AF00000000000000000C18303030303030180CD9
:10AF100000000000000030180C0C0C0C0C0C183059
:10AF2000000000000000000000663CFF3C660000DE
:10AF300000000000000000000018187E1818000033
:10AF400000000000000000000000000000181818B9
:10AF50003000000000000000000000FE00000000C3
:10AF600000000000000000000000000000001818B1
:10AF7000000000000000000002060C183060C080D5
:10AF8000000000000000386CC6C6D6D6C6C66C38B5
:10AF90000000000000001838781818181818187EDB
:10AFA0000000000000007CC6060C183060C0C6FE21
:10AFB0000000000000007CC606063C060606C67CB3
:10AFC0000000000000000C1C3C6CCCFE0C0C0C1EA5
:10AFD000000000000000FEC0C0C0FC060606C67CE3
:10AFE0000000000000003860C0C0FCC6C6C6C67CB9
:10AFF000000000000000FEC606060C18303030309D
:10B000000000000000007CC6C6C67CC6C6C6C67C62
:10B010000000000000007CC6C6C67E0606060C784E
:10B0200000000000000000001818000000181800C0
:10B030000000000000000000181800000018183080
:10B0400000000000000000060C18306030180C06EC
:10B050000000000000000000007E00007E000000F4
:10B06000000000000000006030180C060C18306072
:10B070000000000000007CC6C60C18181800181844
:10B08000000000000000007CC6C6DEDEDEDCC07C06
:10B0900000000000000010386CC6C6FEC6C6C6C65A
:10B0A000000000000000FC6666667C66666666FC62
:10B0B0000000000000003C66C2C0C0C0C0C2663CC8
:10B0C000000000000000F86C6666666666666CF854
:10B0D000000000000000FE6662687868606266FE3C
:10B0E000000000000000FE6662687868606060F042
:10B0F0000000000000003C66C2C0C0DEC6C6663A62
:10B10000000000000000C6C6C6C6FEC6C6C6C6C64B
:10B110000000000000003C18181818181818183CF7
:10B120000000000000001E0C0C0C0C0CCCCCCC78E9
:10B13000000000000000E666666C78786C6666E6E3
:10B14000000000000000F06060606060606266FE09
:10B15000000000000000C6EEFEFED6C6C6C6C6C68B
:10B16000000000000000C6E6F6FEDECEC6C6C6C67B
:10B170000000000000007CC6C6C6C6C6C6C6C67CA7
:10B18000000000000000FC6666667C60606060F0A5
:10B190000000000000007CC6C6C6C6C6C6D6DE7C5F
:10B1A0000C0E00000000FC6666667C6C666666E657
:10B1B0000000000000007CC6C660380C06C6C67CD5
:10B1C0000000000000007E7E5A1818181818183C5D
:10B1D000000000000000C6C6C6C6C6C6C6C6C67CFD
:10B1E000000000000000C6C6C6C6C6C6C66C381041
:10B1F000000000000000C6C6C6C6D6D6D6FEEE6C5D
:10B20000000000000000C6C66C7C38387C6CC6C6E6
:10B21000000000000000666666663C181818183CBE
:10B22000000000000000FEC6860C183060C2C6FE9A
:10B230000000000000003C30303030303030303C16
:10B240000000000000000080C0E070381C0E060204
:10B250000000000000003C0C0C0C0C0C0C0C0C3C16
:10B260000000000010386CC6000000000000000064
:10B2700000000000000000000000000000000000CE
:10B2800000FF000030301800000000000000000047
:10B29000000000000000000000780C7CCCCCCC76D4
:10B2A000000000000000E06060786C666666667C06
:10B2B0000000000000000000007CC6C0C0C0C67CCA
:10B2C0000000000000001C0C0C3C6CCCCCCCCC76FC
:10B2D0000000000000000000007CC6FEC0C0C67C6C
:10B2E000000000000000386C6460F060606060F096
:10B2F00000000000000000000076CCCCCCCCCC7C60
:10B300000CCC78000000E060606C7666666666E6ED
:10B310000000000000001818003818181818183C11
:10B320000000000000000606000E060606060606DF
:10B3300066663C000000E06060666C78786C66E6EB
:10B340000000000000003818181818181818183CC9
:10B35000000000000000000000ECFED6D6D6D6C6E5
:10B36000000000000000000000DC6666666666669D
:10B370000000000000000000007CC6C6C6C6C67CF7
:10B38000000000000000000000DC66666666667C67
:10B390006060F000000000000076CCCCCCCCCC7C0F
:10B3A0000C0C1E000000000000DC7666606060F09F
:10B3B0000000000000000000007CC660380CC67C65
:10B3C000000000000000103030FC30303030361CFF
:10B3D000000000000000000000CCCCCCCCCCCC762F
:10B3E00000000000000000000066666666663C180B
:10B3F000000000000000000000C6C6D6D6D6FE6CD5
:10B40000000000000000000000C66C3838386CC630
:10B41000000000000000000000C6C6C6C6C6C67E0A
:10B42000060CF8000000000000FECC183060C6FEDC
:10B430000000000000000E18181870181818180ED8
:10B440000000000000001818181800181818181824
:10B45000000000000000701818180E181818187056
:10B4600000000000000076DC00000000000000008A
:10B470000000000000000000000066666666667E50
:10B48000626060C0000000000000000000000000DA
:10B4900000000000000000000000000000000000AC
:10B4A000000000000000000000000000000000009C
:10B4B000000000000000000000000000000000008C
:10B4C000000000000000000000000000000000007C
:10BE8000000000000001FF000000000000000000B2
:10BE900000FF010000007A440000FA4300007A43EA
:10BEA0000000C842000048420000C8410000204194
:10BEB0000000A040000020400000803F0000003F44
:10BEC0000000803E04020300536176696E67200023
:10BED0004661696C656431004661696C6564320075
:10BEE0004661696C656433004661696C6564340061
:10BEF0004C6F6164696E670054465420436F6E74E2
:10BF0000726F6C6C65723A0041444320496E7075E3
:10BF1000743A0000497373756520436F64653A0095
:10BF2000542E532E20416D703A20302E3156000091
:10BF3000542E532E20416D703A20332E335600007C
:10BF4000566D61783A000000566D696E3A00000047
:10BF5000566176723A0000005670703A0000000098
:10BF600056726D733A000000467265713A00000027
:10BF70004379636C3A00000050573A004475747975
:10BF80003A000000202500002D2D2D2D000000007E
:10BF9000487A00004B487A004D487A0047487A00BA
:10BFA000730000006D730000757300006E73000075
:10BFB000EFFF0131DFFF0232BFFF03337FFF0434A5
:10BFC000EEFF0535DEFF0636BEFF07377EFF083879
:10BFD0006FFF09415FFF0A423FFF0B439EFF0D4485
:10BFE000F7FF1050F6FF115100000000CDCC4C3D82
:10BFF0000000003E0000803E0000003F0000A03F27
:10C00000000020400000A040000048410000C8415E
:10C01000000048420000FA4200007A430000FA4360
:10C0200000409C4400401C4500409C450050434655
:10C030000050C346005043470024F447002474488E
:10C040000024F448809698498096184A4C69627298
:10C0500061726965732F53544D3332463130785FC6
:10C060005374645065726970685F44726976657272
:10C070002F7372632F6D6973632E63004C69627254
:10C0800061726965732F53544D3332463130785F96
:10C090005374645065726970685F44726976657242
:10C0A0002F7372632F73746D3332663130785F751E
:10C0B000736172742E6300004C696272617269650B
:10C0C000732F53544D3332463130785F537464507C
:10C0D00065726970685F4472697665722F73726306
:10C0E0002F73746D3332663130785F666C617368BC
:10C0F0002E630000737172740000000043000000A2
:10C100000100000008000020000000000000000006
:10C11000000000000000000000000000000000001F
:10C120000000000000000000FCC00008000000004B
:10C1300000000000000000000000000000000000FF
:10C1400000000000000000000000000000000000EF
:10C1500000000000000000000000000000000000DF
:10C1600000000000000000000000000000000000CF
:10C1700000000000000000000000000000000000BF
:10C1800000000000000000000000000000000000AF
:10C19000000000000000000000000000000000009F
:10C1A000000000000000000000000000000000008F
:10C1B000000000000000000000000000000000007F
:10C1C000000000000000000000000000000000006F
:10C1D000000000000000000000000000000000005F
:10C1E000000000000000000000000000000000004F
:10C1F000000000000000000000000000000000F847
:10C20000FCFEFFFEFCF81F3F7FFF7F3F1F0000008A
:10C21000F80000200800070000000000F8181818B7
:10C220005A3C1818181F1F1818183C5A181818F8D4
:10C230001C01002008000A000000000088A4A1A042
:10C24000E5A7BCE58F9C80E591A0A6ADE592929212
:10C25000EB8F9C809180868DEB868A88A08CA08C49
:10C26000A08CA08CA08CA08CA08CA08CA08CA08C6E
:10C27000A08C090009000900090009000900090053
:10C28000090009000900090009000900409C803EDE
:10C29000401FA00F400620039001A000500028007E
:10C2A0001000007D803E0019800C40068002400195
:10C2B000A000400020001000100010003031323388
:10C2C00034353637383941424344454630313233CC
:10C2D00034353637383961626364656600000000C2
:10C2E00064AC00084000220008001000F8A3000819
:10C2F00088000E0088000E0060A500088800150068
:10C300008800150084AE0008080010000800102006
:10C31000E8A4000848000D0048000D00E0AB00084C
:10C3200058000C0058000C00F4A90008700023000D
:10C3300070002300D8A700087800240078002400AB
:10C34000C8A6000890000F0090000F0090BF0008E2
:10C3500094BF000898BF00089CBF0008A0BF000859
:10C36000A4BF0008A8BF0008ACBF0008000001007F
:10C370000200030004000500060007000800090091
:10C380000A000B000C000D000E000F001000110041
:10C3900012001300140015001600170018001900F1
:10C3A000000000000204060800000000010203046F
:08C3B00001020304060708095D
:0400000508000110DE
:00000001FF
